S024000062696E2F6F70656E626C745F6F6C696D65785F73746D3332653430372E737265639F
S315080000000000022059020008A7020008A9020008F9
S31508000010AB020008AD020008AF02000800000000AD
S31508000020000000000000000000000000B102000807
S31508000030B302000800000000B5020008B702000875
S31508000040BB020008BD020008BF020008C102000882
S31508000050C3020008C5020008C7020008C902000852
S31508000060CB020008CD020008CF020008D102000822
S31508000070D3020008D5020008D7020008D9020008F2
S31508000080DB020008DD020008DF020008E1020008C2
S31508000090E3020008E5020008E7020008E902000892
S315080000A0EB020008ED020008EF020008F102000862
S315080000B0F3020008F5020008F7020008F902000832
S315080000C0FB020008FD020008FF0200080103000801
S315080000D003030008050300080703000809030008CE
S315080000E00B0300080D0300080F030008110300089E
S315080000F0130300081503000817030008190300086E
S315080001001B030008353C00081F03000821030008EC
S31508000110230300082503000827030008290300080D
S315080001202B0300082D0300082F030008393C00089C
S3150800013033030008350300083703000839030008AD
S315080001403B0300083D0300083F030008410300087D
S31508000150430300084503000847030008490300084D
S315080001604B0300084D0300084F030008510300081D
S3150800017053030008550300085703000859030008ED
S315080001805B0300085D03000810B5054C237833B9F6
S31508000190044B13B10448AFF300800123237010BD4C
S315080001A00003002000000000FC960008084B10B56C
S315080001B01BB108490848AFF300800848036803B92B
S315080001C010BD074B002BFBD0BDE81040184700BFF9
S315080001D00000000004030020FC960008C00200206E
S315080001E000000000154B002B08BF134B9D46A3F5D6
S315080001F0803A00218B460F461348144A121A08F013
S31508000200D8FD0F4B002B00D098470E4B002B00D083
S3150800021098470020002104000D000D48002802D050
S315080002200C48AFF3008008F06BFD2000290003F0AE
S3150800023087FF08F051FD00BF0000080000000220FB
S31508000240000000000000000000030020A430002089
S31508000250000000000000000007498D460749084ACB
S31508000260084B9A42BEBF51F8040B42F8040BF8E754
S3150800027005488047054800470000022008970008FF
S3150800028000000020C0020020BD0C0008E50100089F
S315080002903349344A002301E041F8043B9142FBD339
S315080002A003F04EFFFEE7FEE7FEE7FEE7FEE7FEE7A2
S315080002B0FEE7FEE7FEE7FEE7FEE7FEE7FEE7FEE708
S315080002C0FEE7FEE7FEE7FEE7FEE7FEE7FEE7FEE7F8
S315080002D0FEE7FEE7FEE7FEE7FEE7FEE7FEE7FEE7E8
S315080002E0FEE7FEE7FEE7FEE7FEE7FEE7FEE7FEE7D8
S315080002F0FEE7FEE7FEE7FEE7FEE7FEE7FEE7FEE7C8
S31508000300FEE7FEE7FEE7FEE7FEE7FEE7FEE7FEE7B7
S31508000310FEE7FEE7FEE7FEE7FEE7FEE7FEE7FEE7A7
S31508000320FEE7FEE7FEE7FEE7FEE7FEE7FEE7FEE797
S31508000330FEE7FEE7FEE7FEE7FEE7FEE7FEE7FEE787
S31508000340FEE7FEE7FEE7FEE7FEE7FEE7FEE7FEE777
S31508000350FEE7FEE7FEE7FEE7FEE7FEE7FEE700004C
S3150800036000030020A430002010B504461346C4F844
S315080003703C21C4F83821022280F811210A460021BE
S3150800038001F0DCF9002010BD08B513460A46002125
S3150800039001F0D4F9002008BD08B513460A46002125
S315080003A001F09EF9002008BD10B50446042380F824
S315080003B0113100231A46194601F0C0F9204601F00A
S315080003C081FE002010BD00BF10B50446052380F845
S315080003D0113100231A46194601F082F9204601F028
S315080003E071FE002010BD00BF0369024A12685A60F8
S315080003F000207047041B002010B50446D0F8E835E5
S315080004001B699847032384F81231002010BD00BFEA
S3150800041008B590F8123180F81331042380F81231A8
S31508000420D0F8E835DB689847002008BD08B5D0F84D
S31508000430E435DB6903B19847002008BD08B5D0F854
S31508000440E4351B6A9847002008BD00BF08B5D0F8F8
S31508000450E4355B6A9847002008BD00BF10B504461E
S31508000460D0F8E8355B699847012384F815310020F0
S3150800047010BD00BF10B50446D0F8E8359B6998470B
S31508000480D4F8E4355B68002120469847002084F8B4
S31508000490150110BD10B5044600234022194601F087
S315080004A0D3F8002340228021204601F0CDF801230D
S315080004B084F81231D4F8E8355B68A07898470020AC
S315080004C010BD00BF10B582B00446694600F02EF98B
S315080004D09DF8001001F01F03012B08D013B1022B61
S315080004E00AD00EE06946204600F094FA0EE0694606
S315080004F0204600F0B3FA09E06946204600F0CAFA39
S3150800050004E001F08001204601F03CF9002002B029
S3150800051010BD00BF10B50446002947D190F8113127
S31508000520022B38D1D0F83821D0F824319A4211D983
S31508000530D21AC0F83821C178012904D1D0F8281177
S315080005400B44C0F8283192B2D4F828112046FFF798
S315080005501BFF20E0D0F83C11B1FBF3F203FB1212AB
S3150800056062B98B420AD8D0F84031994206D2114670
S31508000570FFF70AFF0023C4F840310CE0D4F8E4354D
S31508000580DB682BB194F81221032A01D1204698473B
S315080005902046FFF719FF94F81631012B11D1204692
S315080005A0FFF722FF002384F816310AE00A46D0F83E
S315080005B0E4355B692BB190F81211032901D1114674
S315080005C09847002010BD00BF10B5044659BB90F8E7
S315080005D01131032B32D1D0F89033D0F87C239342D3
S315080005E014D99B1AC0F89033C178012904D1D0F8E0
S315080005F080131144C0F880139A4228BF1A4692B253
S31508000600D4F880132046FFF7C7FE17E0D0F8E43584
S315080006101B6923B190F81221032A00D19847204676
S31508000620FFF7C2FE0AE00A46D0F8E4359B692BB10B
S3150800063090F81211032901D111469847002010BDE0
S31508000640F8B504460D4616461F4603F09BFDC4F84A
S31508000650E475069BC4F8E835C4F8EC6529462046D7
S3150800066000F0A4FFD4F8E8351B689847204603F045
S31508000670E1FDF8BD10B50446D0F8E4351B68984787
S31508000680D4F8E8359B689847002010BD08B5D0F81F
S31508000690E4355B689847002008BD00BF0346002084
S315080006A002E00130C0B201331A78002AF9D1704746
S315080006B010B504464B88012B09D1C0F81831D0F87B
S315080006C0E4359B6898472046FFF76EFE10BD022B5F
S315080006D029D18B8813F0FF0F25D1026952681B0AAE
S315080006E0013B042B17D8DFE803F003070B0F1300B1
S315080006F0012363F306120EE0022363F306120AE0EF
S31508000700032363F3061206E0042363F3061202E0EA
S31508000710052363F30612044B1A60012384F8163185
S315080007202046FFF741FE10BD041B002090F8CC358B
S315080007300B7090F8CD354B7090F8CE3590F8CF25E4
S3150800074003EB02234B8090F8D03590F8D12503EBC4
S3150800075002238B8090F8D23590F8D32503EB022339
S315080007609BB2CB80C0F84031012380F81131704725
S3150800077010B50446802101F005F80021204601F055
S3150800078001F8204601F09EFC10BD00BF30B583B0CD
S3150800079005460C464A88130A013B062B67D8DFE84C
S315080007A003F004162266665E6200D0F8EC351B6814
S315080007B00DF1060180789847E388402B03D095F819
S315080007C01231012B57D10823ADF8063053E0D0F883
S315080007D0E4359B6A0DF10601807898470223437039
S315080007E0C5F8F00547E0D2B2052A34D8DFE802F0AA
S315080007F0030B131B232BD0F8EC355B680DF10601B0
S315080008008078984737E0D0F8EC359B680DF10601FB
S31508000810807898472FE0D0F8EC35DB680DF10601B3
S315080008208078984727E0D0F8EC351B690DF106016A
S31508000830807898471FE0D0F8EC355B690DF1060122
S315080008408078984717E0D0F8EC359B690DF10601DA
S31508000850807898470FE02146FFF78AFF19E021467E
S31508000860FFF786FF15E02146FFF782FF11E02146D4
S31508000870FFF77EFF0DE0BDF8063053B1E28842B1BE
S315080008809A4228BF1A46ADF8062001462846FFF7C1
S315080008906BFD03B030BD00BF38B504468B88E3B99D
S315080008A0CB88D3B98D7805F07F0590F81231032BE4
S315080008B002D1FFF75DFF38BD80F81451294600F0D4
S315080008C0A5FF2046FFF770FD1DB1022384F81231FB
S315080008D038BD012384F8123138BD2046FFF748FF9A
S315080008E038BD00BF10B504468B78214A1370012B1A
S315080008F002D9FFF73DFF10BD90F81221022A02D057
S31508000900032A10D030E05BB180F81031032280F85A
S3150800091012211946FFF7AEFE2046FFF745FD10BD2A
S31508000920FFF742FD10BD5BB9022280F8122180F85C
S3150800093010311946FFF7AAFE2046FFF735FD10BD10
S3150800094090F810118B420CD0FFF7A0FE084B1978CF
S3150800095084F810112046FFF78DFE2046FFF724FD88
S3150800096010BDFFF721FD10BDFFF702FF10BD00BF48
S315080009702003002008B5CB88012B02D0FFF7F8FE2C
S3150800098008BD90F81231022B02D0032B05D00AE0DD
S3150800099001220649FFF7E8FC08BD012200F5887127
S315080009A0FFF7E2FC08BDFFF7E3FE08BD28030020B9
S315080009B008B590F81231023B012B0DD80122084BDD
S315080009C01A60D0F8183113B10322054B1A600222B7
S315080009D00349FFF7C9FC08BDFFF7CAFE08BD00BFFB
S315080009E01C03002010B5044690F81231023B012B77
S315080009F00DD84B88012B0CD10023C0F81831D0F83C
S31508000A00E4359B6898472046FFF7CEFC10BDFFF7F4
S31508000A10AFFE10BD08B54B78092B1BD8DFE803F0ED
S31508000A2011171A141A08051A0E0BFFF7AFFE13E072
S31508000A30FFF732FF10E0FFF755FF0DE0FFF79AFFCB
S31508000A400AE0FFF7B5FF07E0FFF732FE04E0FFF71D
S31508000A50C9FF01E0FFF78CFE002008BD38B5044643
S31508000A600D4690F81231032B0FD10B79012B09D8BB
S31508000A70D0F8E4359B689847EB8843B92046FFF7DA
S31508000A8093FC04E0FFF774FE01E0FFF771FE002017
S31508000A9038BD00BF38B505460C468A88D1B263789A
S31508000AA0012B27D0002B49D0032B40F0818090F8EA
S31508000AB01231022B02D0032B07D017E0002977D07A
S31508000AC0802975D000F05EFE72E0638823B919B1FB
S31508000AD0802901D000F056FED5F8E4359B682146FA
S31508000AE0284698472846FFF75FFC61E02146FFF74E
S31508000AF03FFE5DE090F81231022B02D0032B07D09F
S31508000B0018E0002954D0802952D000F03BFE4FE06F
S31508000B106388002B4CD149B1802907D000F054FED8
S31508000B20D5F8E4359B682146284698472846FFF7B6
S31508000B303BFC3DE02146FFF71BFE39E090F81231F9
S31508000B40022B02D0032B06D02FE089B380292FD0A1
S31508000B5000F018FE2CE052B2002A10DA01F07F01EC
S31508000B6001EB8101CB00034493F81E311BB101222E
S31508000B70104B1A6013E000220E4B1A600FE0002A91
S31508000B800DDB01EB8101CB00034493F876331BB1EF
S31508000B900122084B1A6002E00022064B1A60022264
S31508000BA004492846FFF7E0FB02E02146FFF7E0FD8F
S31508000BB0002038BD24030020D0B170B50D46164676
S31508000BC00446FFF76BFD0130400080B23080287084
S31508000BD003236B70022307E05A1CD2B20134E9548E
S31508000BE00233DBB20021A95421780029F4D170BD63
S31508000BF0704700BFFEE700BF82B000230193009351
S31508000C002A4A136843F480331360284B1B6803F49D
S31508000C1000330093019B01330193009B1BB9019B91
S31508000C20B3F5A06FF1D1214B1B6813F4003F02D036
S31508000C300123009301E000230093009B012B32D18E
S31508000C401A4B1A6C42F080521A6419490A6842F41F
S31508000C5040420A609A689A609A6842F400429A602A
S31508000C609A6842F4A0529A60124A5A601A6842F088
S31508000C7080721A600D4B1B6813F0007FFAD040F2A1
S31508000C8005620D4B1A60A3F580639A6822F0030289
S31508000C909A609A6842F002029A60044B9B6803F0D5
S31508000CA00C03082BF9D102B0704700BF0038024088
S31508000CB0007000400C544007003C024010B5104C30
S31508000CC0D4F8883043F47003C4F888300D4B1A689A
S31508000CD042F001021A60002199601A6822F08472B3
S31508000CE022F480321A60084A5A601A6822F480226E
S31508000CF01A60D960FFF780FF4FF00063A36010BD4C
S31508000D0000ED00E0003802401030002430B585B010
S31508000D1004460D46038A9BB223F44053CA881343FC
S31508000D20038283899BB223F4B05323F00C01A8886D
S31508000D302A896B89024313430B43A381A38A9BB277
S31508000D4023F44073AA891343A382684600F0AEF9D8
S31508000D50204B9C4203D003F580639C4201D1039A41
S31508000D6000E0029AA38913F4004F08D002EB82022E
S31508000D7002EB820229684900B2FBF1F107E002EBB7
S31508000D80820202EB820229688900B2FBF1F1124B5A
S31508000D90A3FB01235B091B011A09642000FB12123D
S31508000DA0A18911F4004F08D0D20032320A49A1FBBA
S31508000DB00212C2F342121A4307E0120132320649FE
S31508000DC0A1FB0212C2F343121A4392B2228105B062
S31508000DD030BD00BF001001401F85EB5129B1838942
S31508000DE09BB243F400538381704783899BB223F4F3
S31508000DF000539BB283817047C1F308018180704715
S31508000E008088C0F3080070470388194201D0012082
S31508000E1070470020704700BF014B1860704700BF3D
S31508000E20DC00274208B501214FF4006000F0E0F924
S31508000E3000214FF4006000F0DBF908BD10B40B4C3C
S31508000E40636823F4FD4121F07F01027D83681A431C
S31508000E5043681A43C3681A43036813430269134372
S31508000E600B4363605DF8044B704700BF002C0140DC
S31508000E70014B1860704700BFA0802542014B1860DF
S31508000E80704700BF002C0140024B186800F00300B1
S31508000E90704700BF002C014010B40368094CA360DA
S31508000EA0E36823F4FF6121F00701426883681A4367
S31508000EB0C3681343026913430B43E3605DF8044BAD
S31508000EC0704700BF002C0140014B1869C0B270473B
S31508000ED0002C014082B000230193034B0344019385
S31508000EE0019B186802B07047142C014010B40368BF
S31508000EF009494B6243688B62CB6A23F0F704826820
S31508000F00C3681A4303691343426913432343CB62F5
S31508000F105DF8044B704700BF002C0140014BD3F825
S31508000F2080007047002C0140014BC3F880007047D1
S31508000F30002C0140034B5B6B034201D00120704734
S31508000F4000207047002C0140014B9863704700BF92
S31508000F50002C0140054B1B69002B05DA034B044A9C
S31508000F605A6002F188325A60704700BF003C02405E
S31508000F7023016745024A136943F00043136170472A
S31508000F80003C0240014BD860704700BF003C02405D
S31508000F900E4BDB6813F4803F10D10C4BDB6813F063
S31508000FA0100F0DD1094BDB6813F0EF0F0AD1074B71
S31508000FB0DB6813F0020F07D007207047012070473F
S31508000FC0052070470620704708207047003C0240FD
S31508000FD000B583B008238DF80730FFF7D9FF8DF8E1
S31508000FE0070003E0FFF7D4FF8DF807009DF80730E8
S31508000FF0DBB2012BF6D09DF8070003B05DF804FBC1
S3150800100070B5054631B1012906D0022907D14FF43A
S31508001010007606E0002604E04FF4807601E04FF4FF
S315080010204076FFF7D5FF08281ED1104C236923F414
S315080010304073236123691E432661236923F0F8035D
S31508001040236123691D4345F002052561236943F49D
S3150800105080332361FFF7BCFF236923F00203236172
S31508001060236923F0F803236170BD00BF003C0240EA
S3150800107070B505460E46FFF7ABFF082813D10A4C94
S31508001080236923F440732361236943F400732361BE
S31508001090236943F0010323612E60FFF799FF236953
S315080010A023F00103236170BD003C024010B4294BB4
S315080010B09B6803F00C03042B05D0082B06D053BB02
S315080010C0254B036029E0254B036026E0214B5A682F
S315080010D05B6803F03F0312F4800F09D01F4AB2FB86
S315080010E0F3F21C4B5B68C3F3881303FB02F208E0B8
S315080010F0194AB2FBF3F3174A5168C1F3881101FB89
S3150800110003F2144B5B68C3F3014301335B00B2FB84
S31508001110F3F3036001E0104B03600E4CA368C3F3BE
S3150800112003130F49CB5CDAB20368D3404360A26865
S31508001130C2F382228A5CD2B223FA02F28260A268E1
S31508001140C2F342328A5CD2B2D340C3605DF8044B24
S31508001150704700BF003802400024F400001BB700A7
S315080011603000002021B1054B1A6B104318637047F5
S31508001170024A136B23EA00001063704700380240E6
S3150800118021B1054B5A6B104358637047024A536B9B
S3150800119023EA0000506370470038024021B1054B2E
S315080011A01A6C104318647047024A136C23EA00004D
S315080011B0106470470038024021B1054B5A6C104341
S315080011C058647047024A536C23EA0000506470471B
S315080011D00038024021B1054B1A691043186170475F
S315080011E0024A136923EA000010617047003802407A
S315080011F021B1054B5A6A104358627047024A536A2E
S3150800120023EA0000506270470038024070B4002399
S315080012103AE001229A400C68A24334D104685D0082
S315080012200322AA40D2431440046006680C79AC40F5
S31508001230344304600C79013CE4B2012C15D8846867
S315080012402240826084684A79AA40224382604668BE
S315080012509AB20124944026EA0404446046688C79CC
S3150800126004FA02F292B232434260C4689AB2560055
S315080012700322B24024EA0202C260C668CC7904FAA4
S3150800128005F23243C26001330F2BC2D970BC7047D6
S315080012900369194201D0012070470020704700BF3A
S315080012A030B401F007039B009A40C908083150F88A
S315080012B021400F2505FA03F324EA030340F82130F9
S315080012C050F821301A4340F8212030BC704700BF3F
S315080012D00A4B0B4A9A6000221A60DB605A60402269
S315080012E05A719A884FF4C86161F30C029A80802279
S315080012F0DA7041F20C0203498B507047801C0020BB
S31508001300901C002000800240054B064A9A60DB606C
S3150800131000221A605A6041F2100203498B50704746
S3150800132080290020D0220020008002402DE9F041CB
S31508001330B2B001214FF0F050FFF714FF012147200A
S31508001340FFF710FF01214FF48040FFF735FF01201A
S31508001350FFF762FD8E23309300258DF8C6500224D0
S315080013608DF8C4408DF8C7508DF8C5405B4F30A93D
S315080013703846FFF74BFF0B2201213846FFF790FF4F
S315080013800B2221463846FFF78BFF0B2203213846EE
S31508001390FFF786FF0B2207213846FFF781FF4FF438
S315080013A0006330938DF8C6508DF8C4408DF8C75049
S315080013B08DF8C54007F5C05730A93846FFF726FF10
S315080013C00B2211463846FFF76BFF322330938DF810
S315080013D0C6508DF8C4408DF8C7508DF8C540DFF863
S315080013E00C8130A94046FFF711FF0B220121404628
S315080013F0FFF756FF0B2204214046FFF751FF0B2249
S3150800140005214046FFF74CFF4FF4C04330938DF853
S31508001410C6508DF8C4408DF8C7508DF8C54030A920
S315080014203846FFF7F3FE0B220D213846FFF738FF43
S315080014300B220E213846FFF733FF01F073F901F04E
S315080014408DFB01F093FB0128FBD001A801F076F98A
S315080014500025019508954FF400730B930C954FF0F2
S3150800146000430F93202312931495159516954FF460
S31508001470006309934FF48043069313E0ACB202214C
S31508001480204601F0ABF960F31F460321204601F020
S31508001490A5F960F30F06124B9E4205D0114B9E42EA
S315080014A002D001351F2DE9D9202D04D94FF4A17199
S315080014B00D4802F0D5FEA9B201A801F0EDF920B950
S315080014C040F24711084802F0CBFEFFF71DFFFFF771
S315080014D0FFFE01F089FB32B0BDE8F0810000024052
S315080014E019162200F1C00700F48D00080008024012
S315080014F0064B08221A7000225A7027229A7069220F
S31508001500DA705B221A7145225A717047941A0020C4
S3150800151038B50D4BDB7813F0800F13D10A4D688868
S31508001520C0F30D0422460949094807F037FCEB7851
S3150800153043F08003EB70012141F20803054AD150BC
S31508001540204638BD002038BD801C0020901C002095
S31508001550602A00200080024038B50F4BDB7813F074
S31508001560800FFAD10D4B1C880D4D22460D49284691
S3150800157007F014FC084B9D6000221A601021997030
S315080015805A60C4F30B049C80B022DA70012141F240
S315080015900403054AD15038BD80290020D0290020EF
S315080015A0D0220020602A00200080024038B5044678
S315080015B000F0A0F9012384F81231002284F81421DE
S315080015C015E091001144CB002344012183F81D1135
S315080015D083F81C21A3F82221002183F81F1140203B
S315080015E0C3F82401C3F82811C3F830110132607812
S315080015F08242E6D3002214E091001144CB00234432
S31508001600002183F8751383F87423A3F87A2383F8E3
S3150800161077134025C3F87C53C3F88013C3F888139F
S3150800162001328242E8D3204600F01EFA204600F036
S31508001630CBF90021204600F063FA204600F0AEFA06
S31508001640204600F009FA38BD70B54DB2002D09DA0A
S3150800165001F07F0606EB8606F40004F58C74044454
S31508001660043408E001F07F0606EB8606F40004F56C
S315080016705C740444043401F07F012170ED0F657039
S31508001680A260E37005B1E180022B01D1002323712A
S31508001690214600F041FB002070BD00BF10B54AB2DC
S315080016A0002A09DA01F07F0404EB8404E30003F559
S315080016B08C730344043308E001F07F0404EB8404CC
S315080016C0E30003F55C730344043301F07F011970EA
S315080016D0D20F5A70194600F051FB002010BD00BF0A
S315080016E070B501F07F04A6003519E9000D4601F52D
S315080016F05C71014404310544C5F88023C5F8883374
S315080017000023C5F88C3385F8753385F87443C37898
S31508001710012B05D104EB8405EB000344C3F88423AD
S3150800172004EB8404E300034493F8743313B900F01C
S31508001730E7FB01E000F046FB002070BD70B501F044
S315080017407F05AE007119CC0004F58C740444211D84
S315080017502E44F4000444012684F81D6184F81C51C3
S31508001760C4F82821C4F82C210022C4F83421C4F86E
S31508001770303115B900F0C4FB01E000F023FB00206E
S3150800178070BD00BF10B54AB2002A09DA01F07F041D
S3150800179004EB8404E30003F58C730344043306E086
S315080017A001EB8104E30003F55C730344043301246D
S315080017B09C7001F07F011970D20F5A70194600F01B
S315080017C033FC002010BD00BF10B54AB2002A09DA62
S315080017D001F07F0404EB8404E30003F58C730344EF
S315080017E0043306E001EB8104E30003F55C7303446C
S315080017F0043300249C7001F07F011970D20F5A70CF
S31508001800194600F02DFC204610BD00BF002361F3E9
S315080018100A13026911680B431360704708B5036918
S31508001820596841F002025A60032002F011FD08BD12
S31508001830C3684FF0FF325A60C3686FF080425A613E
S31508001840014BC268936170470008008030B583B0C9
S31508001850054600240194032002F0EEFCEB681A69A1
S31508001860019201340E4A944217D8019A002AF2DAF4
S31508001870019A42F001020192019A1A610023EA686C
S31508001880126901920133064A934203D8019A12F06B
S31508001890010FF4D1032002F0CFFC002003B030BDC5
S315080018A0400D030010B4C4786CB903339B10323270
S315080018B000EB82008468002203E051F8040B2060E4
S315080018C001329A42F9D300205DF8044B704700BFF5
S315080018D010B403329210D0F8D040002303E02068F9
S315080018E041F8040B01339342F9D308465DF8044BDB
S315080018F0704700BF30B40023C370012383704023B0
S31508001900838001290DD10123C372082303700423A0
S3150800191043704FF4A073C380022303724FF0A044B0
S315080019200CE051B90023C3720C23037006234370DD
S315080019304FF4A063C380234C00E00024C46004F580
S315080019400063036100230FE004EB431202F5106500
S31508001950191D00EB81018D6002F5306203F1140157
S3150800196000EB81014A60013342789342ECD304F5D7
S315080019708063436104F58863C0F8CC30002309E02E
S3150800198004EB431101F5A06103F1220200EB820288
S31508001990916001330578AB42F2D3002309E004EBEA
S315080019A0033101F5805103F1320200EB82029160A6
S315080019B00133AB42F3D304F56064C0F80C41002050
S315080019C030BC70470000044038B50446037A012B42
S315080019D022D10025C268936B6FF31043417A09B18F
S315080019E043F480139363E268D3686FF386136FF347
S315080019F096536FF351436FF3D343D3602046FFF7F3
S31508001A0025FFE378012B19D1052363F3440545F037
S31508001A102005E3689D6011E0C268D16841F0400383
S31508001A20D360FFF713FF4FF45023627A0AB14FF4DD
S31508001A30E813E2689363142002F00AFCE378012BAA
S31508001A4007D1E3689D68052262F3440545F0200541
S31508001A509D60002038BD00BFC268936843F001034B
S31508001A6093600020704700BFC268936823F00103A3
S31508001A7093600020704700BF00B583B00023019330
S31508001A80019A42F020020192019A61F38A120192A8
S31508001A90C26801991161C268126901920133074A45
S31508001AA0934203D8019A12F0200FF4D1032002F0D2
S31508001AB0C3FB002003B05DF804FB00BF400D030024
S31508001AC000B583B000230193019A42F010020192F7
S31508001AD0C26801991161C268126901920133074A05
S31508001AE0934203D8019A12F0100FF4D1032002F0A2
S31508001AF0A3FB002003B05DF804FB00BF400D030004
S31508001B0008B5C268D3686FF35D736FF39E730129D6
S31508001B1002D143F0005302E009B943F08043D36091
S31508001B20322002F095FB002008BD00BFC368586943
S31508001B3000F00100704700BF08B5FFF7F7FF10F186
S31508001B40FF3018BF012008BDC36858699B69184053
S31508001B50704700BF0269136861F301031360704799
S31508001B6038B505460024C3689C61C3686FF0804297
S31508001B705A61FFF75DFEEB7803B9102444F0804400
S31508001B8044F4701444F4605444F00C04EA6893690D
S31508001B9023EA04031C439461002038BD70B504464B
S31508001BA00025D0F80C311D600269136865F3CC2353
S31508001BB01360C37A012B27D12E460321FFF7CAFFEC
S31508001BC0E26880235362202262F31F4563F30F0500
S31508001BD0E1688D62A02161F30F0663F31F46E3688F
S31508001BE0C3F804614FF4907363F30F0662F31F465C
S31508001BF0E368C3F808614FF4A07363F30F066FF345
S31508001C001F46E368C3F80C6110212046FFF734FF2E
S31508001C102046FFF755FF236900221A6123695A6196
S31508001C2023694FF0FF3199612369DA6116E0131DC4
S31508001C3004EB83039B681B68002B02DA4FF0904184
S31508001C4000E00021131D04EB83039868016099687E
S31508001C50002008619B68FF219960013263789A42E7
S31508001C60E5D3002218E002F1140304EB83035B6852
S31508001C701B68002B02DA4FF0904100E0002102F1C8
S31508001C80140304EB8303586801605968002008614F
S31508001C905B68FF219960013263789A42E3D322692F
S31508001CA0136943F480731361E378012B09D1032385
S31508001CB0402262F38A0343F4803362F3594322696C
S31508001CC013632046FFF74CFF002070BD03699B682D
S31508001CD0C3F34103022B04D005D8012B03D00320FC
S31508001CE07047012070470220704700BF03699B6850
S31508001CF082691168C3F34103022B02D06FF30A010C
S31508001D0002E0032363F30A0111600269536843F48E
S31508001D10807353600020704730B400224B78012B43
S31508001D2008D10D782C1D00EB8404A468AB4063F33E
S31508001D300F0209E00D7805F1140400EB84046468C9
S31508001D400123AB4063F31F42236813F4004F0DD100
S31508001D508D6865F30A03CD7865F39343C98861F303
S31508001D60995343F0805343F4004323600369D969C8
S31508001D700A43DA61002030BC704700BF70B4002205
S31508001D8015464B78012B08D10E78311D00EB8101E1
S31508001D908C68B34063F30F0509E00B7803F114046C
S31508001DA000EB840464680121994061F31F456FF3D1
S31508001DB0CF3222600269D36923EA0503D361002082
S31508001DC070BC704738B54B78012B58D10B78043363
S31508001DD000EB83039B681A681C694B692BB96FF380
S31508001DE01204012363F3DC440DE063F312048D68E7
S31508001DF02B44013BB3FBF5F363F3DC44CB78012BAF
S31508001E0001D163F35E740B78043300EB83039B689C
S31508001E101C61C378012B07D10B78043300EB8303CD
S31508001E209B680C695C610CE0CB78012B09D04B6987
S31508001E303BB10C78012303FA04F405696B6B234361
S31508001E406B63CB78012B09D103699B6813F4807FF8
S31508001E5002D142F0005201E042F0805242F00442C0
S31508001E600B78043300EB83039B681A60CB78012B4D
S31508001E7044D18B8A0A78C968FFF714FD3EE00B78CF
S31508001E80143300EB83035B681A681C694B6933B922
S31508001E908B6863F31204012363F3DC440CE08D685A
S31508001EA02B44013BB3FBF5F3C3F3090363F3DC44AB
S31508001EB005FB03F363F312040B78143300EB830377
S31508001EC05B681C61C378012B06D10B78143300EBD1
S31508001ED083035B680C695C61CB78012B06D14B796F
S31508001EE013B142F0005201E042F0805242F004423F
S31508001EF00B78143300EB830043681A60002038BD62
S31508001F0030B482B04B78012B49D183691A681C69B1
S31508001F1000944C696CB99DF800406FF306048DF87F
S31508001F2000409DF80240012565F3C4048DF802407F
S31508001F3017E08D68AC4207D94D619DF8004065F3FE
S31508001F4006048DF8004005E09DF8005064F3060588
S31508001F508DF800509DF80240012565F3C4048DF8FC
S31508001F600240009C1C61C478012C06D10C7804340C
S31508001F7000EB8404A4680D69656142F004421A60A6
S31508001F80C378002B4CD14B69002B49D00A78012322
S31508001F9003FA02F201694B6B13434B6340E00B787B
S31508001FA0143300EB83035B681A681B6900934B695B
S31508001FB073B98C689DF8003064F306038DF8003019
S31508001FC09DF80230012464F3C4038DF802300EE054
S31508001FD08C684C619DF8003064F306038DF8003078
S31508001FE09DF80230012464F3C4038DF802300B789F
S31508001FF0143300EB83035B68009C1C61C378012BD8
S3150800200006D10B78143300EB83035B680C695C61BB
S3150800201042F004420B78143300EB830043681A60DD
S31508002020002002B030BC70474B78012B0DD10B78DD
S31508002030043300EB830082681368002B01DA43F04F
S31508002040804343F40013136008E00B78143300EB65
S3150800205083004268116841F400131360002070473A
S315080020604B78012B05D10B78043300EB830080688D
S3150800207004E00B78143300EB8300406802686FF3C2
S315080020805552CB78023BDBB2012B01D842F0805285
S3150800209002600020704700BF03699869DB69184031
S315080020A0000C7047143100EB81014B689A6803698C
S315080020B058691040704700BF03699869DB69184082
S315080020C080B2704782B000230093C0238DF8033096
S315080020D04FF00003012262F3C4038DF8023018237F
S315080020E08DF80030436D009A1A61C378012B08D128
S315080020F0436D00F2CC525A61436D1A684FF0802244
S315080021001A6002B0704700BF10B50446044B1B683E
S315080021105B6A98474FF08043E2685361012010BD1F
S315080021200000002038B50446C3685D6815F0040F42
S3150800213003D0044B1B689B6A9847E3685D600120DF
S3150800214038BD00BF0000002010B50446837A43B1AD
S31508002150D0F80C316FF341036FF30003D0F80C216C
S3150800216013602269536823F001035360054B1B680B
S315080021709B69204698474FF00043E2685361012067
S3150800218010BD00BF0000002030B583B0054600240E
S315080021908DF8074090F812318DF80730154B1B68FB
S315080021A05B6998472B699A684FF40064EB685C6131
S315080021B0AB7AE3B112F0010F19D095F81531012B5E
S315080021C015D19DF80730DBB2032B10D1D5F80C21B9
S315080021D0136843F001031360D5F80C21136843F024
S315080021E003031360044A136943F0060313610120CD
S315080021F003B030BD0000002000ED00E010B5044635
S31508002200044B1B68DB6898470823E2685361012082
S3150800221010BD00BF0000002010B50446044B1B6823
S31508002220DB6998474FF48013E2685361012010BDBB
S315080022300000002010B50446044B1B681B6A98472B
S315080022404FF40013E2685361012010BD000000201E
S3150800225010B402691469536BCB40DB01DBB223432C
S31508002260043100EB81008268906818405DF8044BE1
S31508002270704700BF2DE9F0410746FFF70DFF0446FA
S31508002280002553E014F0010F4ED05FFA85F8414659
S315080022903846FFF707FF064610F0010F2BD0012638
S315080022A005F1140307EB83035B689E60FB78B34272
S315080022B010D105F1140307EB83035B681969AA00BB
S315080022C02A44D3003B44D3F87C23C1F31201521AA3
S315080022D0C3F88C23184B1B681B6841463846984739
S315080022E0FB78012B07D135B997F81131052B02D1A7
S315080022F03846FFF7E7FE16F0020F06D0022605F16C
S31508002300140307EB83035B689E6016F0080F0BD077
S31508002310094B1B689B6838469847082605F114033D
S3150800232007EB83035B689E6001356408002CA9D11E
S315080023300120BDE8F08100BF000000202DE9F04132
S3150800234007460D468A000A44D3000344D3F83021D1
S31508002350D3F83411521AD3F824319A4200D81346C6
S3150800236003F103084FEA98082B1D07EB83039B68C4
S315080023709B6927E05B1A05EB8501CA003A44D2F847
S315080023802461B34200D81E4606F103084FEA9808AE
S31508002390AB002B44DC003C44B3B2EAB2D4F82811B3
S315080023A03846FFF77FFAD4F828313344C4F8283181
S315080023B0D4F834311E44C4F834612B1D07EB83036B
S315080023C09B689B699BB298450BD2AB002B44DA00FD
S315080023D03A44D2F83411D2F83031994201D2002B5E
S315080023E0C8D10120BDE8F0812DE9F0410746FFF785
S315080023F063FE044600265EE014F0010F59D05FFA2A
S3150800240086F841463846FFF723FF054610F0010FC8
S315080024101ED0012303FA06F039694A6B22EA000244
S315080024204A631D46321D07EB820292689360244B6D
S315080024301B685B68414638469847FB78AB4207D12C
S3150800244036B997F81131042B02D13846FFF73AFE10
S3150800245015F0080F05D00825331D07EB83039B6885
S315080024609D6015F0100F05D01025331D07EB83036B
S315080024709B689D6015F0400F05D04025331D07EB7E
S3150800248083039B689D6015F0020F05D00225331D56
S3150800249007EB83039B689D6015F0800F09D03146D2
S315080024A03846FFF74BFF8025331D07EB83039B68F0
S315080024B09D6001366408002C9ED10120BDE8F0819C
S315080024C0000000202DE9F0410546C268936923F013
S315080024D010039361C3681C6A04F00F06C4F34343F0
S315080024E0022B02D0062B1CD02BE047F6F0732342B2
S315080024F027D0C4F30A144FEA860808EB0603DF0060
S3150800250007442246D7F88013FFF7E2F9D7F8803355
S315080025102344C7F88033D7F88C331C44C7F88C4358
S315080025200FE0082200F2CC51FFF7D2F9C4F30A14DF
S31508002530B2009119CB002B44D3F88C231444C3F86A
S315080025408C43EA68936943F0100393610120BDE860
S31508002550F08100BF2DE9F84304460025A8462F461A
S315080025602E460269536823F0010353602946FFF794
S3150800257083FA2B460CE01A1D04EB82029268FF21AF
S31508002580916003F1140204EB8202526891600133F0
S3150800259062789342EFD323694FF0FF329A614FF086
S315080025A0010969F30F0569F31F452369DD6148F0E1
S315080025B00B082369C3F8148047F00B0723691F61CA
S315080025C0226913686FF30A1313602046FFF77AFD32
S315080025D046F48056E3685E61034B1B681B69204618
S315080025E098474846BDE8F8830000002038B50446F9
S315080025F0FFF77CFBE368DD682046FFF767FB0328E7
S3150800260008D10023A3704FF40073A380092363F352
S315080026108D2506E00123A3704023A380052363F3D9
S315080026208D25E368DD604FF40053E26853610120AD
S3150800263038BD00BF2DE9F8430546FFF77DFA0028A7
S315080026406AD02846FFF780FA0646002868D0C0F305
S31508002650074818F0080F04D02846FFF70BFE044673
S3150800266000E0002418F0040F03D02846FFF7BCFE4C
S315080026700443F7B217F0020F02D00223EA68536147
S315080026804FEA166919F0800F03D02846FFF75CFD5C
S315080026900443C6F3072616F0080F03D02846FFF7AB
S315080026A073FD044317F0080F03D02846FFF7A6FD6D
S315080026B0044317F0100F03D02846FFF703FF04431F
S315080026C016F0100F03D02846FFF744FF044316F010
S315080026D0200F03D02846FFF789FF044318F0100F90
S315080026E003D02846FFF798FD044318F0200F03D0BF
S315080026F02846FFF79FFD044319F0400F03D02846EC
S31508002700FFF702FD044317F0040F08D02846FFF729
S3150800271009FD2043BDE8F8830020BDE8F88320467C
S31508002720BDE8F88308B501214FF00070FEF752FDA9
S3150800273000214FF00070FEF74DFD08BD0023036031
S3150800274043608360C360036143618361C36103625D
S3150800275043628362C362036343638363C363402242
S315080027600264202242648364C36403654365836507
S31508002770C3650366802242668366C366036743674A
S315080027808367C3674FF08062C0F880204FF00072FD
S31508002790C0F884204FF08071C0F888104FF40011FB
S315080027A0C0F88C10C0F89030C0F89430C0F8983053
S315080027B0C0F89C30C0F8A030C0F8A420C0F8A830F3
S315080027C04FF40032C0F8AC204FF48072C0F8B02045
S315080027D0C0F8B430C0F8B830704700BF82B00023E4
S315080027E00193124A136903F01C03C00280B2034323
S315080027F0890101F4F8610B4343F001031361019B5E
S3150800280001330193094B1B6913F0010F03D0019A99
S31508002810074B9A42F3D9019A064B9A4203D0034BC7
S31508002820586980B200E0002002B07047008002407C
S31508002830FEFF0400FFFF040010B483B000230193D9
S31508002840124C236903F01C03C00280B203438901BA
S3150800285001F4F8610B4343F0030362612361019BB2
S3150800286001330193094B1B6913F0010F03D0019A39
S31508002870074B9A42F3D9019A064B9A4201D1002096
S3150800288000E0012003B05DF8044B70470080024069
S31508002890FEFF0400FFFF040070B586B004460D462F
S315080028A0002305930093924B1E6926F01C0601A887
S315080028B0FEF7FCFB029A8F4B13448F498B4202D8D2
S315080028C046F008060EE08D4B13448D498B4202D81C
S315080028D046F00C0606E08B4B13448B4A934201D90B
S315080028E046F00406824B1E614FF40042002128463A
S315080028F0FFF7A2FF0646002800F0F7804FF0806336
S31508002900059302E0059B013B0593059E002EF9D130
S315080029102368002B4CD0009B0133009301212846E5
S31508002920FFF75CFF00F0040080B218B9009A774BF5
S315080029309A42F0D9009A764B9A4200F0D680002146
S3150800294000914FF480522846FFF776FF002800F0E2
S31508002950CB80009B0133009301212846FFF73EFFF9
S3150800296000F0200080B218B9009A684B9A42F0D954
S31508002970009A674B9A4200F0B88000230093102112
S315080029802846FFF72BFF00F004039BB21BB14FF458
S315080029900063236201E00023236200F002039BB276
S315080029A013B1002363611CE04FF48043636118E0B0
S315080029B0226AC2F3CF026369C3F34F031A430021A5
S315080029C02846FFF739FF0646002800F08E806FF08C
S315080029D07F43059302E0059B013B0593059B002B6E
S315080029E0F9D1434B1A684B4911406068A2681043F5
S315080029F0E26810432269104362691043A2691043D2
S31508002A00E2691043226A1043626A1043A26A1043BD
S31508002A10E26A1043226B1043626B02430A431A6050
S31508002A20A16BE26B1143226C1143626C1143A26CD9
S31508002A301143E26C1143226D1143626D0A435A60D9
S31508002A40A26D9A60E26DDA609A694FF6417111409B
S31508002A50206E626E42EA0040A26E1043E26E104398
S31508002A60226F1043626F02430A439A61A16FE26FB5
S31508002A700A43DA6141F218055A5927491140D4F830
S31508002A808000D4F884201043D4F888201043D4F862
S31508002A908C201043D4F890201043D4F89420104387
S31508002AA0D4F898201043D4F89C201043D4F8A020DA
S31508002AB002430A435A51D4F8A410D4F8A820114363
S31508002AC0D4F8AC201143D4F8B0200A43D4F8B41093
S31508002AD042EA8101D4F8B8200A4342F4000203F519
S31508002AE080531A60012600E00646304606B070BDDF
S31508002AF00080024000D3CEFEBFE1E40040F1E9FDCC
S31508002B003F787D0100796CFC005A6202FEFF0400E2
S31508002B10FFFF04000F8120FF233FDEF828B1064A95
S31508002B20136843F0080313607047034A136823F0D9
S31508002B3008031360704700BF0080024028B1064AA8
S31508002B40136843F0040313607047034A136823F0BD
S31508002B5004031360704700BF00800240024A1368EE
S31508002B6043F001031360704700900240044B1B6852
S31508002B7013F0010F01D0012070470020704700BFF5
S31508002B8000900240034941F218028B5843F480131F
S31508002B908B5070470080024038B1084941F218024C
S31508002BA08B5843F400538B507047044941F218027E
S31508002BB08B5823F400538B50704700BF00800240A7
S31508002BC038B1084941F218028B5843F002038B507A
S31508002BD07047044941F218028B5823F002038B50C0
S31508002BE0704700BF0080024008B50120FFF796FF36
S31508002BF0FFF7C8FF0120FFF7A1FF0120FFF7CCFF71
S31508002C000120FFF7DDFF08BD2DE9F04182B0012163
S31508002C100C20FEF7A7FA2C4C0C2208212046FEF7BA
S31508002C203FFB0C2209212046FEF73AFB0C220A211B
S31508002C302046FEF735FB0C220B212046FEF730FB1B
S31508002C400C2211462046FEF72BFB204F0C220221B0
S31508002C503846FEF725FB4FF47063009301258DF87F
S31508002C6005504FF002088DF8048000268DF806609E
S31508002C708DF8075069462046FEF7C8FA04230093E4
S31508002C8069463846FEF7C2FA4FF4805300938DF82A
S31508002C90076069462046FEF7B9FA4FF400670097C1
S31508002CA08DF804808DF8076069462046FEF7AEFA6F
S31508002CB029463846FEF780FA29464FF48000FEF783
S31508002CC051FA02B0BDE8F08100080240000C02404B
S31508002CD010B54FF4803400E0013C24B18020FEF7A3
S31508002CE029F90028F8D02CB140F2FF50FEF72CF94C
S31508002CF0002010BD032010BD08B5104B5A6B4FF4C9
S31508002D00803302E0013B0D4A526B12F0450F01D1A8
S31508002D10002BF7D113B112F0040F04D00420FEF7EC
S31508002D2013F9032008BD12F0400F04D04020FEF727
S31508002D300BF9002008BD002008BD00BF002C01408B
S31508002D4008B50B4B5B6B01E0094B5B6B13F0450F4A
S31508002D50FAD013F0040F04D00420FEF7F5F8032088
S31508002D6008BD40F2FF50FEF7EFF8002008BD00BF8F
S31508002D70002C014008B50F4B5B6B01E00D4B5B6BFC
S31508002D8013F0450FFAD013F0040F04D00420FEF711
S31508002D90DBF8032008BD13F0010F04D00120FEF76D
S31508002DA0D3F8012008BD40F2FF50FEF7CDF8002009
S31508002DB008BD00BF002C014010B50446444B5B6BB0
S31508002DC001E0434B5B6B13F0450FFAD013F0040F89
S31508002DD004D00420FEF7B8F8032010BD13F0010F45
S31508002DE004D00120FEF7B0F8012010BDFEF76CF8FC
S31508002DF0A04243D140F2FF50FEF7A6F80020FEF7A6
S31508002E0069F8344B0340DBB300283BDB10F0804FF6
S31508002E103AD110F0005F39D110F0805F38D110F048
S31508002E20006F37D110F0806F36D110F0807F35D122
S31508002E3010F4000F34D110F4800F33D110F4001FB2
S31508002E4032D110F4801F31D110F4002F30D110F494
S31508002E50802F2FD110F4003F2ED110F4803F2DD1B2
S31508002E6010F4004F2CD110F4804F2BD110F4005FD2
S31508002E702AD110F0080F29D01A2010BD102010BD35
S31508002E80002010BD1C2010BD092010BD0A2010BD51
S31508002E900B2010BD0C2010BD0D2010BD0E2010BD3E
S31508002EA00F2010BD102010BD112010BD122010BD1E
S31508002EB0132010BD142010BD152010BD162010BDFE
S31508002EC0172010BD182010BD192010BD002010BDF8
S31508002ED0002C014008E0FFFD38B504460D461E4BA0
S31508002EE05B6B01E01C4B5B6B13F0450FFAD013F0DC
S31508002EF0040F04D00420FEF727F8032038BD13F08A
S31508002F00010F04D00120FEF71FF8012038BDFDF798
S31508002F10DBFFA04218D140F2FF50FEF715F800205B
S31508002F20FDF7D8FF10F4604F03D1000C288000206D
S31508002F3038BD10F4005F09D110F4804F08D110F4A1
S31508002F40004F07D00F2038BD102038BD132038BDDC
S31508002F50102038BD002038BD002C0140F0B583B0E4
S31508002F600E46002300930193564808220260102457
S31508002F70446040228260C3604FF480630361FDF7BA
S31508002F808BFF2046FFF718FF002840F094804E4B31
S31508002F901B68A3404B480360372444604023836082
S31508002FA00023C3604FF480630361FDF775FF204675
S31508002FB0FFF702FF00287FD144484FF0FF33036034
S31508002FC008234360302383600223C360002404611E
S31508002FD001234361FDF78AFF3A48046033254560BB
S31508002FE040238360C4604FF480630361FDF754FF98
S31508002FF02846FFF7E1FE054600285ED127460EE083
S315080030004FF40010FDF796FF20B1FDF787FF4DF846
S3150800301027000137013442F210739C424ED82C4BDC
S315080030205A6B40F22A631A42EAD00820FDF782FF5B
S3150800303020B10820FDF788FF042040E00220FDF7B4
S3150800304079FF20B10220FDF77FFF022037E020201C
S31508003050FDF770FF20B12020FDF776FF06202EE051
S315080030604FF40070FDF766FF28B14FF40070FDF7C6
S315080030706BFF072023E040F2FF50FDF765FF00993C
S315080030800B0203F47F0343EA01630A0A02F47F4250
S31508003090134343EA1163736001990B0203F47F0338
S315080030A043EA01630A0A02F47F42134343EA1163BF
S315080030B03360284603E002E001E000E0042003B0A4
S315080030C0F0BD00BFE803002088030020300300207D
S315080030D0002C014010B582B00446002000900190F3
S315080030E0FDF7F8FE10F0007F5CD16946324B188870
S315080030F0FFF734FF002857D1012C2AD1019B13F47E
S31508003100802F52D02C4B1B681B042C480360372495
S315080031104460402383600023C3604FF480630361E7
S31508003120FDF7BAFE2046FFF747FE00283FD12348A1
S315080031300223036006244460402383600023C3609F
S315080031404FF480630361FDF7A7FE2046FFF734FEC0
S3150800315030E0019B13F4803F2AD0174B1B681B04F1
S315080031601648036037244460402383600023C36005
S315080031704FF480630361FDF78FFE2046FFF71CFEC0
S31508003180C0B90E48002303600624446040228260CA
S31508003190C3604FF480630361FDF77EFE2046FFF7A8
S315080031A00BFE07E00E2005E004E0252002E001E022
S315080031B02520FFE702B010BD88030020E8030020A1
S315080031C000B583B001238DF807304FF40061064837
S315080031D0FEF75EF810B900238DF807309DF8070052
S315080031E003B05DF804FB00BF0008024070B582B06A
S315080031F000248DF80740664876230375046044600A
S315080032008460C4600461FDF719FE0320FDF736FEED
S315080032100120FDF72DFE5F48046044608460C460A9
S315080032204FF480630361FDF737FEFFF751FD8DF814
S3150800323007009DF8073013F0FF0F03D09DF807002D
S31508003240C0B2A3E053484FF4D57303600823436024
S31508003250402383600023C3604FF480630361FDF756
S315080032601BFEFFF749FD8DF807009DF8073013F0A0
S31508003270FF0F05D10122484B1A604FF0804611E036
S315080032804448002606603724446040238360C660AD
S315080032904FF480630361FDF7FFFD2046FFF78CFDC1
S315080032A08DF807003B48002303603724446040221A
S315080032B08260C3604FF480630361FDF7EDFD20462D
S315080032C0FFF77AFD8DF807009DF8073013F0FF0F1A
S315080032D040D058E02F480023036037254560402238
S315080032E08260C3604FF480630361FDF7D5FD28460D
S315080032F0FFF762FD8DF807009DF8073013F0FF0F02
S3150800330003D09DF80700C0B240E046F0004343F4FE
S3150800331080132048036029234360402383600023E9
S31508003320C3604FF480630361FDF7B6FDFFF708FD40
S315080033308DF807009DF8073013F0FF0F03D09DF8AE
S315080033400700C0B222E00020FDF7C4FD0246C00F08
S31508003350013402E000200446024618B94FF6FE730F
S315080033609C42B7D94FF6FE739C4206D91B238DF8AB
S3150800337007309DF80700C0B208E012F0804F02D06F
S315080033800222054B1A609DF80700C0B202B070BD54
S3150800339070030020E80300205803002010B582B00F
S315080033A00123ADF80630FDF76FFD00286AD0394BCA
S315080033B01B68042B20D03848002303600222426091
S315080033C0C0228260C3604FF480630361FDF764FD29
S315080033D0FFF7D0FC002857D1FDF77CFD2F4C206065
S315080033E00420FDF777FD60600820FDF773FDA060F7
S315080033F00C20FDF76FFDE060264B1B68012B03D9F7
S31508003400062B01D0022B12D1234800230360032484
S31508003410446040228260C3604FF480630361FDF715
S315080034203BFD0DF106012046FFF756FD68BB194B1B
S315080034301B68042B2AD0BDF80630194A13601B04F2
S315080034401548036009234360C02383600023C360D3
S315080034504FF480630361FDF71FFDFFF78BFCB8B9D6
S31508003460FDF738FD0F4C20600420FDF733FD606042
S315080034700820FDF72FFDA0600C20FDF72BFDE0606E
S31508003480002005E0252003E002E001E00020FFE738
S3150800349002B010BD58030020E80300205C0300209A
S315080034A08803002048030020F0B40346A44A1468A1
S315080034B080F85640A34A1288A0F85420A24D2A68DC
S315080034C0100EC1B28E091E70C0F38300587001F049
S315080034D003019970C2F30741D970C2F30721197124
S315080034E0D2B25A7169680A0E1201DA80C1F307402E
S315080034F0DA8892B242EA1012DA8000F00F001872E7
S31508003500080AC2B2D5095D72C0F380159D72C0F370
S315080035104015DD72C0F300151D7300255D73012C7F
S3150800352044D8800200F4406018611A69890001F4E1
S315080035307F7111431961844A9268100EC1B21C69E1
S3150800354044EA91141C61C0F3C200187501F0070122
S315080035505975110CC1F342109875C1F38200D875DC
S31508003560490001F006011976C2F30722197E41EADD
S31508003570D21119761C6901349C64DD64187E023008
S31508003580012505FA00F0C717A0FB040104FB071183
S31508003590C3E912011C7AE4B205FA04F41C65A4FB1B
S315080035A0006704FB0177C3E9126721E0022C1FD1EB
S315080035B0090401F47C111961634A9268100E1969AD
S315080035C041EA002119611969C2F3074001431961EB
S315080035D0C2F3072218690021013041F10001C9042C
S315080035E041EA5031C0049864D9644FF400711965F2
S315080035F0C2F380115976520002F07E029A7652483A
S31508003600027A997E41EAD211997602F07F02DA7639
S31508003610C1680A0ED0091877C2F341105877C2F369
S3150800362082009877920002F00C02DA77080CC2B290
S31508003630DC7F44EA9214DC77C0F3401083F820005C
S31508003640002083F8210002F0010283F822200A0AEA
S31508003650D4B2E50983F82350C2F3801583F82450C1
S31508003660C2F3401583F82550C2F3001583F8265097
S31508003670C2F3810283F8272004F0030483F8284064
S31508003680C1F3460183F82910012483F82A402F4DF7
S315080036902A68110E83F82C10C2F307410902D9854E
S315080036A0C2F30726D98D89B23143D98512061A6322
S315080036B06A68160E196B41EA06411963110C1E6BEE
S315080036C0090201F47F4131431963196BC2F30726D6
S315080036D031431963D2B283F83420AA68110E83F8ED
S315080036E03510110C09069963110A9E6B090401F439
S315080036F07F0131439963996B120202F47F420A43B0
S315080037009A63EA68996B41EA12619963110C93F816
S315080037103C60C1F30315354383F83C50090201F4B4
S315080037207061D987C2F30725D98F89B22943D9870A
S31508003730C2F3460283F8402083F84140F0BC704744
S315080037405803002088030020480300205C0300205B
S315080037501C4B1B68032B2CD0022B2CD8B0F5805F92
S315080037602BD010B5B0F5006F12D10120FFF7B2FCCF
S31508003770044620BB14480023037503604360836036
S315080037804FF40062C2600361FDF758FB204610BD86
S315080037900020FFF79FFC044690B90B4800230375E9
S315080037A0036043608360C3600361FDF747FB2046FF
S315080037B010BD27207047002070472720704710BD8E
S315080037C010BD00BF580300207003002010B5094B38
S315080037D0186007245C6040229A600022DA604FF481
S315080037E080621A611846FDF757FB2046FFF7E4FA90
S315080037F010BD00BFE803002000B583B000238DF894
S315080038000730FFF701FAFDF70DFBFFF7EFFC8DF820
S3150800381007009DF8073013F0FF0F03D09DF8070047
S31508003820C0B237E0FFF7BAFD8DF807009DF80730FC
S3150800383013F0FF0F03D09DF80700C0B22AE017481F
S3150800384000230375036043608360C3600361FDF76B
S31508003850F5FA1348FFF728FE8DF807009DF807309C
S3150800386013F0FF0F08D10E4BB3F8540000040021E3
S31508003870FFF7ACFF8DF807009DF8073013F0FF0F30
S3150800388005D14FF40060FFF763FF8DF807009DF838
S315080038900700C0B203B05DF804FB00BF7003002048
S315080038A090030020F8B505461646BDF81810002204
S315080038B05248027052480260524802605248C26238
S315080038C0524A1268022A04D1720A42EAC3564FF4CF
S315080038D000710F464E480160102343604023836001
S315080038E00023C3604FF480630361FDF7D5FA4FF4F4
S315080038F0803400E0013C24B18020FDF71BFB002842
S31508003900F8D01020FFF758FA002874D141484FF034
S31508003910FF3303604760902383600223C360002758
S31508003920076101234361FDF7E1FA3948066011246E
S31508003930446040238360C7604FF480630361FDF7EA
S31508003940ABFA2046FFF738FA064680B154E04FF442
S315080039500040FDF7EFFA50B105E0FDF7DFFA45F84C
S315080039602400013400E00024072CF6D92035264B24
S315080039705A6B40F22A631A42E9D00820FDF7DAFAB0
S3150800398020B10820FDF7E0FA0420F8BD0220FDF773
S31508003990D1FA20B10220FDF7D7FA0220F8BD20207F
S315080039A0FDF7C8FA20B12020FDF7CEFA0620F8BDAB
S315080039B04FF40070FDF7BEFA58B14FF40070FDF7EA
S315080039C0C3FA0720F8BDFDF7A9FA45F8040B013C30
S315080039D001E04FF0FF344FF40010FDF7ABFA08B1E1
S315080039E0002CF0D140F2FF50FDF7AEFA00220A4B48
S315080039F01A603046F8BDF8BDF8BD00BF2C0300209C
S31508003A006C030020FC030020002C01405803002012
S31508003A10E803002030030020400000202DE9F04193
S31508003A2005461646BDF81810002256480270564834
S31508003A300260564802605648C262564A1268022A0E
S31508003A4004D1720A42EAC3564FF400710F4652482F
S31508003A50016010244460402383600023C3604FF450
S31508003A6080630361FDF718FA2046FFF7A5F90028D9
S31508003A7040F08380484806601824446040238360E9
S31508003A800023C3604FF480630361FDF705FA2046FF
S31508003A90FFF792F90446002871D140484FF0FF33EA
S31508003AA003604760902383600026C6600661012391
S31508003AB04361FDF71BFA2AE04FF48040FDF73AFA16
S31508003AC028B3C6F50078B8F11F0F1BD8734213F058
S31508003AD0030F02D14FEA980803E04FEA980808F165
S31508003AE00108002705E055F8040BFDF71DFA013714
S31508003AF004364745F7D30AE055F82700FDF714FAC8
S31508003B00013700E00027072FF6D920352036204B4D
S31508003B105A6B40F21A631A42CED00820FDF70AFA09
S31508003B2028B10820FDF710FA0420BDE8F08102202C
S31508003B30FDF700FA28B10220FDF706FA0220BDE8D3
S31508003B40F0811020FDF7F6F928B11020FDF7FCF9F1
S31508003B500520BDE8F0814FF40070FDF7EBF930B1B0
S31508003B604FF40070FDF7F0F90720BDE8F081002258
S31508003B700B4B1A602046BDE8F081BDE8F081BDE830
S31508003B80F08100BF2C0300206C030020FC030020FA
S31508003B90002C014058030020E803002030030020D1
S31508003BA040000020D8B138B505460E4B1B681B04EB
S31508003BB00D4803600D244460402383600023C360DE
S31508003BC04FF480630361FDF767F92046FFF7F4F8C1
S31508003BD0044630B9FDF77EF92860204638BD262010
S31508003BE0704738BD88030020E803002000B583B07D
S31508003BF000230193FFF7E4FA012807D101A8FFF78C
S31508003C00D1FF28B90198C0F3432002E0FF2000E065
S31508003C10FF2003B05DF804FB08B5FFF7E7FF0428AB
S31508003C2003D0FF2803D1022008BD002008BD0120CB
S31508003C3008BD00BF704700BF704700BF00B597B00A
S31508003C40FFF7DAFD48B9084A137803F0FE03137044
S31508003C506846FFF729FC002003E00122024B1A7090
S31508003C60032017B05DF804FB4400002008B50122C4
S31508003C70064B1A7038B9FFF7CFFF20B9034A1378F5
S31508003C8003F0FE031370014B187808BD44000020AA
S31508003C9070B5ADF5027D0E461546B8B11BE0621942
S31508003CA04FF4007300935202002302A8FFF7FAFDAF
S31508003CB098B9FFF7B1FF0128FBD04FF4007202A9AB
S31508003CC006EB442005F06AF8234644B15C1E002B37
S31508003CD0E5D1012004E0012002E0012000E00020F7
S31508003CE00DF5027D70BD00BFF0B5ADF5037D0F463D
S31508003CF01646C0B11CE04FF400752A4607EB44216E
S31508003D0002A805F04BF8A21900955202002302A852
S31508003D10FFF784FE08B105280CD1FFF77DFF0128BF
S31508003D20FBD0234644B15C1E002BE4D1012004E0FD
S31508003D30012002E0012000E000200DF5037DF0BD22
S31508003D40174B1B7813F0010F1FD103291FD8DFE883
S31508003D5001F00204131800207047D0B910B596B0C8
S31508003D6014466846FFF7A0FB129B5B0A139A43EAC0
S31508003D70C2532360002010E04FF400731380002024
S31508003D80704740B92023136070470320704704200A
S31508003D907047002070470020704716B010BD00BF5E
S31508003DA04400002012230B8000487047680000205A
S31508003DB004230B80004870476400002010B5044CAB
S31508003DC00A4621460348FCF7F7FE204610BD00BF09
S31508003DD0081B0020088E000810B5044C0A46214628
S31508003DE00348FCF7E9FE204610BD00BF081B00206B
S31508003DF01C8E000810B5044C0A4621460348FCF7F9
S31508003E00DBFE204610BD00BF081B00202C8E0008D4
S31508003E1010B5044C0A4621460348FCF7CDFE204659
S31508003E2010BD00BF081B00203C8E000810B5044CCE
S31508003E300A4621460348FCF7BFFE204610BD00BFD0
S31508003E40081B0020448E000820230B80004870477A
S31508003E50A800002008B590F81231032B01D101F013
S31508003E60C5FE002008BD00BF08B501F0BFFE002052
S31508003E7008BD00BF08B5084601F0EAFE002008BDE7
S31508003E8008B50B7813F0600F21D14B780A2B12D0A6
S31508003E900B2B15D0062B1AD14B881B0A212B05D1C3
S31508003EA0CA88172A28BF17220A4901E00A49172291
S31508003EB0FCF75AFA0BE001220849FCF755FA06E026
S31508003EC08B7813B9054A136001E0FCF751FC002012
S31508003ED008BD00BFBA000020B10000200004002081
S31508003EE010B504468121FDF7D9FB01212046FDF7CF
S31508003EF0D5FB002010BD00BF10B5044602234022A2
S31508003F008121FDF7A1FB0223402201212046FDF76E
S31508003F109BFB4023034A01212046FDF7E1FB0020D5
S31508003F2010BD00BF90290020004870479029002046
S31508003F30704700BF704700BF704700BF08B5012132
S31508003F400448FDF7A5F9012801D1002008BD012084
S31508003F5008BD00BF0000024000B5C7B04FF48C7220
S31508003F600021684604F025FF69460A4803F05AFD11
S31508003F7038B9009B3BB19DF8083013F0100F04D0F8
S31508003F8004E0002002E0002000E0012047B05DF8D0
S31508003F9004FB00BF5C8E0008004870475C8E000872
S31508003FA008B50748002380F828320A22054903F095
S31508003FB0BBF918B90122024B83F8282208BD00BFB5
S31508003FC0040400207C8E000810B50D4B93F82832A7
S31508003FD0012B02D10A4803F05FFC01F001F900F158
S31508003FE0640403E001F0FCF8844205D34021054847
S31508003FF0FCF70AFF0028F5D0034803F039FD10BD89
S3150800400004040020001401405C8E000808B5044B27
S3150800401093F82832012B02D1014803F03DFC08BD74
S315080040200404002010B504460F4B93F82832012BE0
S3150800403015D10D4903F0A4FD002810DA0A4800231B
S3150800404080F8283203F028FC09E00848FCF7D4FE7B
S3150800405080210648FCF7D8FE0028F9D001342178DB
S315080040600029F2D110BD00BF04040020001401404D
S31508004070F0B583B0FCF722FE01210846FDF772F879
S315080040800124009400268DF804608DF80760022547
S315080040908DF8055069462848FDF7B8F821462020CE
S315080040A0FDF78AF821460420FDF75CF8234F08221D
S315080040B006213846FDF7F4F8082207213846FDF7A9
S315080040C0EFF88DF806608DF807408DF80450402308
S315080040D000938DF8055069463846FDF797F88DF830
S315080040E004508023009369463846FDF78FF8214629
S315080040F02846FDF737F8A7F58067092205213846CF
S31508004100FDF7CEF8092206213846FDF7C9F86023DF
S3150800411000938DF804508DF805508DF806608DF8DB
S31508004120074069463846FDF771F821464FF0C060EA
S31508004130FDF734F803B0F0BD000002400008024065
S3150800414008B5FFF795FF00F031FC00F03FFCFCE7EF
S31508004150704700BF704700BF704700BF08B5FFF73C
S31508004160E9FE08BD08B5FFF7E7FE08BD08B501205A
S31508004170FFF7DEFE08BD00BF08B50020FFF7D8FE32
S3150800418008BD00BFF0B583B001210846FCF7EAFF79
S315080041904FF4C853009303278DF8057002238DF852
S315080041A0043000268DF806608DF80760204C6946B5
S315080041B02046FDF72BF80A2208212046FDF770F85D
S315080041C00A220B212046FDF76BF80A220C2120460D
S315080041D0FDF766F84FF4007300938DF805708DF8B7
S315080041E0046001258DF806508DF80760694620465B
S315080041F0FDF70CF84FF4806300938DF806508DF8A0
S3150800420007508DF8057069462046FCF7FFFF0A221D
S3150800421011462046FDF744F829464FF48040FCF73E
S31508004220CBFF29468020FCF7ABFF03B0F0BD00BFEB
S3150800423000000240704700BF06E000BF013300E0FF
S3150800424000231B2BF9D91046421E0028F8D17047C7
S3150800425008B54FF47A7303FB00F0FFF7EDFF08BDCE
S3150800426008B500F0A1FBFCE7034601310D4AA2FBA5
S315080042700323DB08F9D110B400230B70094BA3FB09
S315080042800023DB081A4603EB83035C00031B303369
S3150800429001F8013D1046002AF0D108465DF8044BA6
S315080042A0704700BFCDCCCCCC00F00F03092802D94B
S315080042B003F13700704710B503F1300404F052FDDE
S315080042C02044437803F00303022B00D1203CE0B2DC
S315080042D010BD00BF38B505460C460009FFF7E4FFD8
S315080042E0207005F00F00FFF7DFFF60700023A37052
S315080042F0204638BDF8B50746002634461EE0BD5DA3
S3150800430004F030FD2844437803F00303022B00D160
S31508004310203DEBB2A3F13002D2B2162A12D8A3F18D
S315080043203A01C9B206290FD9092A01D9373BDAB2A7
S315080043302301DBB21344DCB20136F6B2012EDED914
S315080043402046F8BD0020F8BD0020F8BD08B50022BB
S31508004350054B1A700549064802F0BAFF18B17721CD
S315080043600448FFF77DFF08BD700600208C8E000804
S315080043707C060020908E0008034B1B780BB90120A1
S3150800438070470020704700BF7006002008B500F08F
S31508004390FFFB01280AD0084B1B784BB9FFF7DCFD59
S315080043A0012807D10122044B1A7008BD002008BD58
S315080043B0002008BD002008BD7006002038B5054657
S315080043C0047804F0CFFC2044437803F00303022B5F
S315080043D000D1203C532C0FD104F0C4FC6B78184450
S315080043E0427812F0040F09D0312B09D0322B09D0AC
S315080043F0332B09D1022038BD032038BD032038BD30
S31508004400002038BD012038BD032038BD70B50646EA
S315080044100230FFF76FFF054684B204363046FFF7D1
S3150800442069FF2844C5B2013CA4B20236012CF5D86E
S31508004430ED43EDB23046FFF75DFF854201D000201F
S3150800444070BD012070BD00BFF8B5044616460F467C
S3150800445001B120B940F261214D48FFF701FF20461E
S31508004460FFF7ACFF0546032800F08A802046FFF7D1
S31508004470CDFF002800F08680012D25D015B1022D2C
S315080044804CD082E0A01CFFF735FF85B2201DFFF750
S3150800449031FF00023860A01DFFF72CFF3B68184467
S315080044A038600834E81E05B24EB92846F8BD2046DD
S315080044B0FFF720FFF05502340137BFB200E00027AE
S315080044C0AF42F4DB2846F8BDA01CFFF713FF85B200
S315080044D0201DFFF70FFF00043860A01DFFF70AFF35
S315080044E03B6803EB0020386004F10800FFF702FF81
S315080044F03B68184438600A34281F05B24EB9284666
S31508004500F8BD2046FFF7F6FEF05502340137BFB274
S3150800451000E00027AF42F4DB2846F8BDA01CFFF7F1
S31508004520E9FE85B2201DFFF7E5FE00063860A01DEE
S31508004530FFF7E0FE3B6803EB0040386004F1080033
S31508004540FFF7D8FE3B6803EB0020386004F10A0049
S31508004550FFF7D0FE3B68184438600C34681F05B274
S315080045604EB92846F8BD2046FFF7C4FEF05502347A
S315080045700137BFB200E00027AF42F4DB2846F8BD9A
S315080045800020F8BD4FF0FF30F8BD0020F8BD00BF91
S31508004590908E000870B5AC4B1B78002B00F0E781B5
S315080045A0012B29D101F080FBFFF7FAFCA748FFF79A
S315080045B039FDA748FFF736FDFFF7EEFC0122014655
S315080045C0A44802F0B1FE30B1A348FFF72BFD012045
S315080045D0FFF71CFD70BDA148FFF724FDA048FFF7B3
S315080045E021FDA048FFF71EFD9F4B00221A605A6066
S315080045F00222954B1A7070BD022B40F0EF809B4C3F
S3150800460004F50C724FF48071994803F08FFA94F808
S3150800461041326BB19048FFF705FD0220FFF7F6FC23
S3150800462004F50C7003F038F90022874B1A7070BD38
S31508004630B0B18F48002200F5C071FFF705FF0446A8
S31508004640B0F1FF3F0DD18448FFF7ECFC0320FFF7DC
S31508004650DDFC804803F020F900227B4B1A7070BD00
S315080046600024002C5BDD804B5B6833B9804BD3F8A4
S3150800467080217D4B1A605C6051E07D4AD2F880113A
S31508004680794A12681A44914203D12344764A536000
S3150800469045E07248FFF7C6FC7648FFF7C3FC764E3E
S315080046A0714D31466868FFF7DFFD3046FFF7BAFC03
S315080046B07248FFF7B7FC3146E878FFF70BFEB11CE6
S315080046C0A878FFF707FE311D6878FFF703FEB11DCE
S315080046D02878FFF7FFFD3046FFF7A4FC6848FFF788
S315080046E0A1FC6968286801F0E7FA60B95A48FFF73B
S315080046F099FC0520FFF78AFC564803F0CDF80022FE
S31508004700514B1A7070BD5548FFF78CFC5548FFF79A
S3150800471089FC574BD3F88021534B1A605C60534B86
S31508004720D3F84422D3F83C329A4240F02081002143
S31508004730484803F0C3F860B14748FFF773FC042004
S31508004740FFF764FC434803F0A7F800223E4B1A70B3
S3150800475070BD454B5B68002B39D04048FFF762FCBB
S315080047604448FFF75FFC444D3F4C29466068FFF715
S315080047707BFD2846FFF756FC4048FFF753FC2946C1
S31508004780E078FFF7A7FDA91CA078FFF7A3FD291D70
S315080047906078FFF79FFDA91D2078FFF79BFD284647
S315080047A0FFF740FC3648FFF73DFC6168206801F0DA
S315080047B083FA60B92848FFF735FC0520FFF726FC81
S315080047C0244803F069F800221F4B1A7070BD23486D
S315080047D0FFF728FC03221C4B1A7070BD032B40F010
S315080047E0C680224C04F50C724FF48071204803F001
S315080047F09DF994F841326BB12248FFF713FC022069
S31508004800FFF704FC04F50C7003F046F800220E4B83
S315080048101A7070BD002839D0154800F5807200F569
S31508004820C071FFF711FE0546B0F1FF3F2FD11648BC
S31508004830FFF7F8FB0320FFF7E9FB064803F02CF81F
S315080048400022014B1A7070BD70060020A88E000861
S31508004850CC8E0008AC080020F48E0008FC8E0008F8
S31508004860048F0008288F0008740600207C060020A4
S31508004870D40A0020588F000830060020648F0008EC
S3150800488008900008808F0008A48F00080025002DD6
S3150800489040DD3748FFF7C6FB364C21462846FFF76A
S315080048A0E3FC2046FFF7BEFB3348FFF7BBFB334E5E
S315080048B0214696F88301FFF70DFDA11C96F88201A3
S315080048C0FFF708FD211D96F88101FFF703FDA11DDD
S315080048D096F88001FFF7FEFC2046FFF7A3FB284861
S315080048E0FFF7A0FB06F580722946D6F8800101F08D
S315080048F0DFF960B92348FFF795FB0620FFF786FB2B
S31508004900214802F0C9FF0022204B1A7070BD2048CA
S31508004910FFF788FB1F4BD3F84422D3F83C329A4260
S3150800492025D11D48FFF77EFB01F0D2F960B915487D
S31508004930FFF778FB0720FFF769FB134802F0ACFF87
S315080049400022124B1A7070BD1148FFF76BFB134813
S31508004950FFF768FB0C4802F09FFF1148FFF762FB60
S3150800496000220A4B1A70FFF72FFB00F0A3FF70BD59
S31508004970C88F000830060020D88F0008D40A002007
S3150800498008900008F48E0008AC0800207006002085
S31508004990FC8E00087C060020F08F00080C900008AA
S315080049A024900008704700BF704700BF08B500F0A4
S315080049B07DFFFFF7F7FF00F0F1FB01F075F9FFF750
S315080049C0C5FC00F041F800F02FF808BD08B5FFF760
S315080049D0EBFF00F0F7FBFFF7DDFD00F04DF800F008
S315080049E001F808BD08B500F0D3F8012817D0FFF77D
S315080049F0C3FCA0B10A4B1B78012B10D100F0F0FBC9
S31508004A00084B1B6803F51C531033984207D3002242
S31508004A10034B1A70FFF7BAFC08B900F04BFF08BD44
S31508004A20580C00205C0C002008B50122044B1A70B3
S31508004A3000F0D6FB034B1860FFF7D4FF08BD00BF94
S31508004A40580C00205C0C002010B500F013FB00F099
S31508004A50FBFB084C0123237001F07AF9002323702D
S31508004A6001F018F80223237000F000F903232370DD
S31508004A7010BD00BFE400002000B583B00DF10701AA
S31508004A801E4800F0EDFC012807D101221C4B1A70C4
S31508004A909DF80710194800F00BFB0DF107011748A0
S31508004AA001F09CF9012807D10022154B1A709DF8D0
S31508004AB00710124800F0FCFA0DF107010F4801F043
S31508004AC04DF8012807D102220D4B1A709DF80710E0
S31508004AD00A4800F0EDFA0DF10701084800F01AF946
S31508004AE0012807D10322064B1A709DF807100348C0
S31508004AF000F0DEFA03B05DF804FB00BF600C00208E
S31508004B00E400002008B500F0F7FF08BD38B50446F4
S31508004B100D46104B1B78012B02D1C9B200F04EFC92
S31508004B200C4B1B781BB9E9B2204601F02FF9094B4B
S31508004B301B78022B03D1E9B2204600F0E7FF054BAC
S31508004B401B78032B03D1E9B2204600F0C5F800F024
S31508004B50A7FA38BDE4000020054B1B78012B05D0C9
S31508004B60022B01D0402070473F207047082070472D
S31508004B70E4000020054B1B78012B05D0022B01D041
S31508004B80402070473F20704708207047E400002007
S31508004B9008B500F07DFA08BD10B5FCF7B9FC48B3B6
S31508004BA02C4A10802C4B9C894FF4006003F024F9A2
S31508004BB084420DD1012003F059F9264B1B88CBB14D
S31508004BC003F0DAFFFCF7C8FC0022224B1A8011E03A
S31508004BD0214B9C8940F6060003F00EF9844209D160
S31508004BE003F05AFF1B4B1B8823B1FCF7B5FC0022C8
S31508004BF0184B1A8000F0F4FA184B1B6898421BD31E
S31508004C0003F5FA73154A1360002413E0144A68235F
S31508004C1003FB0423134A1360022003F027F90D4B04
S31508004C201B8833B103F0A8FFFCF796FC0022094B5A
S31508004C301A800134002CE9D000F0D2FA0A4B1B681E
S31508004C40984206D303F51C531033074A136003F042
S31508004C50F1FE10BDD0290020602A0020A40C0020F7
S31508004C60E8290020E4290020A00C002008B5FCF75C
S31508004C705DFB00F0B5FA00F5FA70124B186000F00B
S31508004C80AFFA00F51C5010300F4B186003F06CF8A3
S31508004C900E4B4FF6A9621A8043F6137159800C4BD6
S31508004CA04FF6FF711980002159800A4B1A8040F28D
S31508004CB013125A804EF6030003F084F8FCF718FC2A
S31508004CC008BD00BFA40C0020A00C00205C2A002010
S31508004CD0582A0020542A002038B50D4B1D68EB6968
S31508004CE02B62002306E01A1DC45C2A4482F8204081
S31508004CF001339BB28AB29342F5D3111DA5F864100D
S31508004D0005F1200003F000FEEB690133EB6138BDC5
S31508004D10E429002008B5FFF73FFF002008BD00BFC3
S31508004D2010B5174B1C68174B1B7813F0400F05D0AE
S31508004D300123E3610023A4F8643010BD13F0010FCA
S31508004D4002D00022A4F8642013F0040F06D0B4F8A9
S31508004D50641019B104F1200003F0D6FD094B1B7845
S31508004D6013F0020F0BD00023A4F86430064B186822
S31508004D70064B19780439C9B2043000F099F910BD08
S31508004D80E4290020DC290020E0290020D029002081
S31508004D900022014B5A707047A80C0020034BFE22D4
S31508004DA0DA7018710222A3F844207047A80C002074
S31508004DB010B5054C00232370FFF7EAFFFF23E370C5
S31508004DC00123A4F8443010BDA80C0020064BFF228E
S31508004DD0DA7000221A71597859719A71DA711A7251
S31508004DE00622A3F844207047A80C002008B5002026
S31508004DF0FFF7D4FF08BD00BF084BFF22DA70084A48
S31508004E009A6400221A715A719A710721D9711A7215
S31508004E105A729A720822A3F844207047A80C0020F8
S31508004E2050900008044BFF22DA7042689A64012207
S31508004E30A3F84420704700BFA80C002008B531200D
S31508004E40FFF7ACFF08BD00BF38B5084CFF23E37079
S31508004E50002525716571FFF77FFEA071E571257242
S31508004E6065720723A4F8443038BD00BFA80C00209B
S31508004E7038B5FFF781FA18B91020FFF78FFF38BD4C
S31508004E80FFF786FF0D4C01252570FF23E3701023DD
S31508004E90237100236371FFF75FFEA071FFF76AFEB7
S31508004EA0E071FFF767FEC0F3072020726572A572EE
S31508004EB00823A4F8443000F0F7FE38BDA80C0020FB
S31508004EC038B505464478FFF747FE0138844203DDC6
S31508004ED02220FFF763FF38BD084C6A78A16C201DB5
S31508004EE000F004FDFF23E3706B78A26C1344A364FF
S31508004EF06B780133A4F8443038BD00BFA80C0020F5
S31508004F0038B504464578FFF727FE0138854203DDA4
S31508004F102220FFF743FF38BD6168084DA96462780F
S31508004F20281D00F0E3FCFF23EB706378AA6C13449A
S31508004F30AB6463780133A5F8443038BDA80C00206B
S31508004F40F8B505461746002406E015F8013B1C444B
S31508004F50E4B2FFF729FD31464E1E0029F5D13C6023
S31508004F600120F8BD10B5084CFF23E370E21D416827
S31508004F70A06CFFF7E5FF207100236371A371082376
S31508004F80A4F8443010BD00BFA80C002038B505466B
S31508004F900D4B9C6CFFF7E0FD6A1C411E204600F095
S31508004FA087FE18B93120FFF7F9FE38BD064CFF23F6
S31508004FB0E370FFF7D1FD0138A36C1844A064012300
S31508004FC0A4F8443038BD00BFA80C002038B5044604
S31508004FD04578FFF7C1FD0238854203DD2220FFF739
S31508004FE0DDFE38BD0F4BFF22DA700122A3F84420FC
S31508004FF0617831B900F06CFE90B93120FFF7CEFE2A
S3150800500038BDA21C074B986C00F052FE18B9312027
S31508005010FFF7C4FE38BD6378024A916C0B4493646B
S3150800502038BD00BFA80C002008B54168074B986C2E
S3150800503000F042FE18B93120FFF7B0FE08BD034B59
S31508005040FF22DA700122A3F8442008BDA80C00202C
S3150800505008B500F02FFC034BFF22DA700122A3F8F3
S31508005060442008BDA80C002008B589B2FFF74EFDFC
S3150800507008BD00BF054B00221A709A6483F84320C6
S31508005080A3F844209A705A70704700BFA80C0020F5
S31508005090024B187800B10120704700BFA80C002009
S315080050A00022024B83F84320704700BFA80C00205B
S315080050B008B50378FF2B02D1FFF7DAFE50E0334A32
S315080050C01278012A60D1C93B352B46D8DFE803F0B0
S315080050D03345454245453F363C39454545454545B1
S315080050E04545454545454545454545454545454562
S315080050F045454545454545454545241E1B214545E8
S315080051004527452A2D30FFF7DBFE29E0FFF7F8FE95
S3150800511026E0FFF787FE23E0FFF724FF20E0FFF7EE
S315080051206BFE1DE0FFF762FE1AE0FFF74FFE17E081
S31508005130FFF73EFE14E0FFF729FF11E0FFF746FFF1
S315080051400EE0FFF781FE0BE0FFF76EFF08E0FFF7C2
S315080051507FFF05E0FFF772FE02E02020FFF71EFE44
S315080051600A4B93F84330012B02D11020FFF716FEA5
S31508005170064BB3F94410002906DD1846012380F8CA
S3150800518043300330FFF770FF08BD00BFA80C0020AE
S315080051900022014B1A60704710E000E008B5FFF7DF
S315080051A0F7FF054B054A5A6000229A6005211960E7
S315080051B0034B1A6008BD00BF10E000E03F900200F4
S315080051C0F40C0020044B1B6813F4803F03D0034AF9
S315080051D0136801331360704710E000E0F40C0020F8
S315080051E008B5FFF7EFFF014B186808BDF40C00205F
S315080051F0F0B5002421E0134D15F8147005EB4405AD
S3150800520095F801E007EB0E0505FB00054AF2104C80
S315080052109CFBF5F605FB16C66EB99CFBF5F5ADB21B
S315080052200D80013DADB2B5F5806F04D2177083F8D5
S3150800523000E00120F0BD0134E4B2112CDBD90020D6
S31508005240F0BD00BF8090000810B582B001AB0DF12B
S3150800525005020DF106014FF4FA70FFF7C9FF0128A0
S3150800526004D040F207115148FEF7FAFF504B0022CE
S315080052705A611A6842F400421A60FFF7B1FF00F15A
S31508005280FA0405E0FFF790FBFFF7AAFF844204D370
S31508005290474B1B6813F4004FF4D1454B1A6822F0AC
S315080052A002021A601A6842F001021A60FFF798FFB4
S315080052B000F1FA0405E0FFF777FBFFF791FF844258
S315080052C004D33B4B5B6813F0010FF4D09DF805300F
S315080052D05A1E9DF80430013B1B0543EA0243BDF8FC
S315080052E00620013A1343324AD361136823F00103B7
S315080052F01360FFF775FF00F1FA0405E0FFF754FBAA
S31508005300FFF76EFF844204D3294B5B6813F0010F45
S31508005310F4D1284BD3F8002242F00102C3F8002248
S31508005320D3F8002222F47C52C3F80022D3F80022D4
S3150800533042F46062C3F80022D3F8002242F0010268
S31508005340C3F80022D3F81C2222F48042C3F81C2298
S31508005350D3F80C2242F48042C3F80C22D3F8042274
S3150800536022F48042C3F80422134AC3F8B02202F199
S315080053704C520432C3F8B422D3F8042222F48042F1
S31508005380C3F80422D3F8142222F48042C3F8142264
S31508005390D3F81C2242F48042C3F81C22D3F8002218
S315080053A022F00102C3F8002202B010BD589000088E
S315080053B000680040006400400000E0CC38B50446B0
S315080053C00D46254B9B6813F0806F04D140F28B1174
S315080053D02248FEF745FF204BD3F8802102F0010250
S315080053E0C3F88021D3F8802142F07C4242F40012AF
S315080053F0C3F88021C3F88451E178A278120442EAFE
S315080054000162617842EA012221780A43C3F88821B9
S31508005410E179A279120442EA0162617942EA01223B
S3150800542021790A43C3F88C21D3F8802142F001027E
S31508005430C3F88021FFF7D4FE00F1320405E0FFF738
S31508005440B3FAFFF7CDFE844204D3034B9B6813F0EF
S31508005450806FF4D038BD00BF00680040589000083F
S31508005460244BDB6813F0030F41D0224BD3F8B0313D
S3150800547013F0040F04D11F4BD3F8B0315B0D05E0D0
S315080054801C4BD3F8B031DB0843F0004340F26762A7
S31508005490934225D1174BD3F8B42102F00F020A70B4
S315080054A0D3F8B8210270D3F8B821120A4270D3F89B
S315080054B0B821120C8270D3F8B821120EC270D3F834
S315080054C0BC210271D3F8BC21120A4271D3F8BC215F
S315080054D0120C8271D3F8BC311B0EC371012000E097
S315080054E00020044AD36843F02003D36070470020A5
S315080054F0704700BF0068004038B50546002419E02B
S31508005500FFF752FA04EB440293000C4AD358AB4215
S315080055100ED804EB44018A0008490A445268134429
S315080055209D4205D204EB440083000B44187A38BD2B
S315080055300134E4B2082CE3D9FF2038BDD490000822
S3150800554008B5C1F3080353B90368994209D040F86E
S31508005550041B4FF4007200F0C9F9012008BD0020B1
S3150800556008BD012008BD00BF2DE9F04107460068C7
S31508005570FFF7C2FFFF282ED0FBF7ECFCF320FBF762
S3150800558001FDFBF705FD012818D1FBF7F3FC002008
S31508005590BDE8F0813E68A30006EB03083B445D685E
S315080055A0FFF702FA29464046FBF762FD08280AD1AA
S315080055B056F824309D4208D1013400E000247F2C9F
S315080055C0E8D9012402E0002400E00024FBF7D2FC1D
S315080055D02046BDE8F0810020BDE8F08138B50D46CB
S315080055E00B4B984207D004460A4B994205D0FFF761
S315080055F0BBFF18B908E0084C00E0054C29462046D0
S31508005600FFF79EFF10B938BD002038BD204638BDCB
S31508005610F80C002000C00008FC0E00202DE9F0411F
S3150800562006460C4617461D4621F4FF7828F0010861
S315080056300368B3F1FF3F04D14146FFF781FF0346F4
S3150800564030B33368984505D041463046FFF7C6FF64
S315080056500646D0B13368E41A34440434FFF7A4F993
S31508005660331DE31AB3F5007F07D308F500713046FA
S31508005670FFF7B4FF064650B1041D17F8013B04F8BE
S31508005680013B013DEAD1012302E0002300E00023AB
S315080056901846BDE8F08100BF884229D838B50446C7
S315080056A00D46022826D90B2926D8FBF753FCF320EA
S315080056B0FBF768FCFBF76CFC012813D1FBF75AFCD7
S315080056C0002038BDFFF770F902210C4B33F814009F
S315080056D0FBF796FC082803D0FBF74CFC002038BDE6
S315080056E00134E4B2AC42EDD9FBF744FC012038BDE5
S315080056F000207047002038BD002038BDA49000085F
S315080057004FF0FF33024A1360024A1360704700BF26
S31508005710FC0E0020F80C002070B54B1E154C241A00
S31508005720A34221D816460D460446FFF7E5FEFF2894
S315080057301CD028190138FFF7DFFEFF2818D024F4FB
S31508005740FF7323F001030C4A934206D12B463246D7
S3150800575021460A48FFF762FF70BD2B4632462146AE
S315080057600748FFF75BFF70BD002070BD002070BDC5
S31508005770002070BDFFFF0F0800C00008F80C0020CD
S31508005780FC0E00204A1E0E4B1B1A9A4212D870B500
S315080057900D460446FFF7B0FE064628190138FFF7FE
S315080057A0ABFEFF2E08D0FF2808D001463046FFF78B
S315080057B073FF70BD00207047002070BD002070BDCB
S315080057C0FFFF0F08114B1B68B3F1FF3F18D000B558
S315080057D083B00E4B59689A681144DA6811441A69FD
S315080057E011445A6911449A691144DA698B185B4263
S315080057F002AA42F8043D04210548FFF78DFF01E09F
S315080058000120704703B05DF804FB00BFF80C0020C8
S3150800581088C100080D4B1A6804331B6813440C4AE8
S31508005820126813440B4A126813440B4A11680B4456
S31508005830043212681A44094B1B681344084A126852
S31508005840D34201D1012070470020704700C00008EC
S3150800585008C000080CC0000810C0000818C00008DE
S3150800586088C1000808B50D4B1B68B3F1FF3F04D08B
S315080058700A48FFF779FE034668B1094B1B68B3F17E
S31508005880FF3F05D00648FFF76FFE034610B902E052
S31508005890012300E00123184608BD00BFF80C0020CC
S315080058A0FC0E00200048704700C0000808B500F04C
S315080058B0E9FA08BD10B500F003FAA0B1FEF73EFB01
S315080058C088B1FFF71FF9FFF763FC00F0FDF920F038
S315080058D0604020F07F00044B186000F0F5F944683A
S315080058E000F0D2FAA04710BD08ED00E070B508E058
S315080058F0461C4D1C0B780370FFF756F822463046B7
S315080059002946531E9CB2002AF2D170BD094B03F1F9
S315080059101801002205E09A745961183318310132CA
S31508005920D2B2002AF7D09A7400225A61014A024B71
S315080059301A60704748110020441100200B4B1B6861
S3150800594073B110B45C69094A146019749860D86018
S3150800595000225A741860013908445860987C01E09E
S31508005960FF2070475DF8044B704700BF44110020C4
S3150800597038B504460D46012804D940F29D1115484C
S31508005980FEF76EFC62002244D300134A13445A7C85
S315080059901B7C9A421AD062002244D3000E4A134452
S315080059A0DA6815705A7C01325A74DA680132DA609C
S315080059B05B689A420CD9084A63001819C100084660
S315080059C0515803461344D960012038BD002038BD1C
S315080059D0012038BD409100084811002008B501464D
S315080059E0024B1878FFF7C4FF08BD00BFFC11002062
S315080059F038B504460D46012804D940F2BF111448AB
S31508005A00FEF72EFC04EB4402D300124A1344587CDA
S31508005A10E0B162002244D3000E4A13449A68127811
S31508005A202A705A7C013A5A749A6801329A605B68FD
S31508005A309A420AD9074A63001819C10008465158FC
S31508005A40034613449960012038BD012038BD00BFC4
S31508005A50409100084811002008B50146024B187805
S31508005A60FFF7C6FF08BD00BF7811002010B5044631
S31508005A70012804D940F2DF110448FEF7F1FB04EBD4
S31508005A804404E300024A1344587C10BD40910008C0
S31508005A904811002030B583B0FFF738FF0F4C40217E
S31508005AA0601CFFF74BFF20700D4D4021681CFFF767
S31508005AB045FF28702378FF2B01D0FF2803D17921D1
S31508005AC00848FEF7CDFB084B0093084B084A01210E
S31508005AD00848FAF7B5FD03B030BD00BFFC11002039
S31508005AE07811002040910008C80000207C000020A2
S31508005AF0480000204012002008B50348FBF78EFE38
S31508005B000020FEF715FA08BD4012002070B50646BB
S31508005B100D463F2903D99A210F48FEF7A1FB2846CF
S31508005B20FFF75CFF012803D09E210B48FEF798FB80
S31508005B3000240CE0FEF738FF305DFFF74FFF012821
S31508005B4003D0A7210448FEF78BFB0134A4B2ABB2FD
S31508005B509C42EFD370BD00BF4091000870B5064661
S31508005B600D461D48FCF766FD1C4B1C788CB91C4875
S31508005B70FFF772FF01282DD1194B1B78013BDBB2C9
S31508005B803E2B27D80122154B1A700022154B1A7086
S31508005B9020E0144B1B78013311481844FFF75CFFCB
S31508005BA00446012813D10F4B1A780132D2B21A7063
S31508005BB00B4B1B789A420CD10B493046FFF796FEE1
S31508005BC00022064B1A70074B1B782B7002E0002444
S31508005BD000E00024204670BD40120020401100203D
S31508005BE000110020411100200111002030B583B0BA
S31508005BF0134B1878FFF73AFF00B30546402800D93B
S31508005C004025002412E00DF107010D4B1878FFF727
S31508005C10EFFE012804D040F227110A48FEF720FBC0
S31508005C209DF80720084B1A550134E4B2A542EAD874
S31508005C302B46054A81210548FBF780FD03B030BD98
S31508005C40FC11002040910008BC11002040120020E1
S31508005C5070B500EB8000C300104A1344B3F88C6398
S31508005C60002410E00E4B1D78FEF75EF9015D28460C
S31508005C70FFF77EFE012804D04FF4A3710948FEF70A
S31508005C80EFFA0134A4B2B442ECD3FEF74DF940233F
S31508005C90024601210148FBF723FD70BD4012002092
S31508005CA0781100204091000808B5FFF729FD08BDC6
S31508005CB008B5FFF731FD08BD08B5FFF763FD08BD58
S31508005CC008B5FFF7A7FD08BD08B5FFF7EBFD08BD4A
S31508005CD008B5FFF777FD034610B1FFF7C3FD034686
S31508005CE0184608BD10B5044680210F48FBF78CF806
S31508005CF0B0B121460C48FBF77FF8FFF771FA00F1BF
S31508005D000A0405E0FEF750FEFFF76AFA844209D353
S31508005D1080210548FBF778F80028F3D0012010BD4C
S31508005D20002010BD002010BD0014014010B5044627
S31508005D3020210648FBF768F8012805D10348FBF738
S31508005D405FF82070012010BD002010BD001401402E
S31508005D5010B584B04FF4614300930023ADF80430C6
S31508005D60ADF80630ADF80830ADF80C300C23ADF8B8
S31508005D700A30054C69462046FAF7C8FF0121204635
S31508005D80FBF72CF804B010BD0014014070B50646A8
S31508005D900D46402903D979210F48FEF761FA2846AE
S31508005DA0FFF7A0FF012803D07D210B48FEF758FA1C
S31508005DB000240CE0FEF7F8FD305DFFF793FF01289D
S31508005DC003D086210448FEF74BFA0134A4B2ABB2DD
S31508005DD09C42EFD370BD00BF6891000870B5244B94
S31508005DE01C78ACB92348FFF7A1FF01283ED1214B07
S31508005DF01B78013BDBB23F2B38D8FFF7F1F91E4B76
S31508005E00186000221D4B1A700122194B1A702DE0DA
S31508005E1006460D46194B1B78013316481844FFF7FA
S31508005E2085FF0446012813D1144B1A780132D2B2E1
S31508005E301A70104B1B789A4215D111493046FFF754
S31508005E4055FD00220A4B1A700C4B1B782B700DE07F
S31508005E50FFF7C6F9084B1B686433984205D9002436
S31508005E60034B1C7002E0002400E00024204670BDAD
S31508005E70341800203C180020381800207D1800200F
S31508005E803D18002072B6704762B6704742780078AF
S31508005E9040EA0220704700BFC278837843EA0222AC
S31508005EA0437843EA0223007840EA0320704700BF9C
S31508005EB00170090A417070470170C1F307234370E6
S31508005EC0C1F307438370090EC170704713462AB1A0
S31508005ED00A78027001300131013BF9D1704700BFE1
S31508005EE001700130013AFBD1704700BF30B4451C40
S31508005EF0037808781B1A013A04D04C1C2846214618
S31508005F00002BF4D0184630BC704700BF00E00130C3
S31508005F1003780BB18B42FAD11846704702394369A8
S31508005F20023B994204D24389806A01FB0300704709
S31508005F300020704770B506460D4601F11A00FFF7B6
S31508005F40A5FF04463378032B05D105F11400FFF7A6
S31508005F509DFF44EA004070BD70B506460C461546DE
S31508005F6091B204F11A00FFF7A3FF3378032B04D18B
S31508005F70290C04F11400FFF79BFF70BD2DE9F041D1
S31508005F8080460F4601F11A00FFF780FF50BB3D78A7
S31508005F9005F03F056B1E03EB430503EB850501265C
S31508005FA0002411E0174B185D3844FFF76FFF36B130
S31508005FB0FE2D1AD828F815000646013503E04FF6D7
S31508005FC0FF73984214D101340C2CEBD93B7813F0AB
S31508005FD0400F10D0FE2D11D8002328F815300120C7
S31508005FE0BDE8F0810020BDE8F0810020BDE8F08121
S31508005FF00020BDE8F0810120BDE8F0810020BDE861
S31508006000F08100BF249200082DE9F84380460F4628
S3150800601091464B730F23CB7200240C73214607F16C
S315080060201A00FFF745FF09F1FF3303EB430603EBBD
S31508006030860625464FF6FF739D4202D038F816505D
S3150800604001360C4B185D29463844FFF731FF0DB968
S315080060504FF6FF7501340C2CECD94FF6FF739D42B1
S3150800606002D038F816300BB949F0400987F8009085
S31508006070BDE8F8832492000870B582B00546164636
S315080060801C460B22FFF722FF052C12D814E0023615
S3150800609000220CE003F0010101EB44045B0814F450
S315080060A0803F03D084F4883484F0210401320F2A17
S315080060B0F0D93388002BEAD1072300E0134604F011
S315080060C00F0202F13001392901D902F137015A1EAE
S315080060D002A8034403F8081C2409EFD17E210346CD
S315080060E0134403F8081C002300E00133934202D24C
S315080060F0E95C2029F9D1591C2B44072A05D802A89E
S31508006100104410F8080C013200E0202018700B46E5
S315080061100729F0D902B070BD0B210023DA0142EA43
S315080061205303027852FA83F3DBB201300139F5D111
S3150800613018467047016821B94FF0FF3316E001325F
S3150800614000E00A4613781F2B01D93A2BF7D13A2BD0
S315080061500BD110B44C1C0B78303B092B08D8A24243
S3150800616009D15BB9013202600AE00023184670477C
S315080061704FF0FF3304E04FF0FF3301E04FF0FF33F9
S3150800618018465DF8044B704738B50C4670B105469D
S3150800619003685BB11A784AB1D9888288914205D1D9
S315080061A05878FDF763FD10F0010F03D00023236034
S315080061B0092038BD2B682360002038BDF8B5C378A0
S315080061C003B30446C66A00F130070123324639464E
S315080061D04078FDF789FDB8B90023E370236AF31AFE
S315080061E0A269934212D2A57808E0A3691E44012346
S315080061F0324639466078FDF777FD013D012DF4D822
S315080062000020F8BD0020F8BD0120F8BD0020F8BD2B
S3150800621070B5C36A8B4212D004460D46FFF7CEFF0F
S31508006220064668B901232A4604F130016078FDF76D
S315080062302FFD10B101264FF0FF35E56200E000267C
S31508006240304670BD10B504460023C3704FF0FF33C7
S31508006250C362FFF7DDFFD8B904F22E20FFF716FE5A
S315080062604AF65523984215D104F16600FFF714FE45
S3150800627020F07F400A4B98420ED004F18200FFF7C7
S315080062800BFE20F07F40064B984207D1002010BD38
S31508006290042010BD032010BD002010BD022010BD33
S315080062A0464154002DE9F04784B00E4617460023B0
S315080062B00B60FFF73FFF051EC0F22C81AA4B53F86F
S315080062C02540002C00F02881346007F0FE0723786B
S315080062D073B16078FDF7CAFC10F0010F08D1002FE2
S315080062E000F01C8110F0040F40F01A81002038E1FC
S315080062F000232370E8B26070FDF7A0FC10F0010FD0
S3150800630040F010811FB110F0040F40F00D810021FC
S315080063102046FFF797FF022815D0002628E004F14B
S3150800632030002B0103F5DF73184403791BB10830DD
S31508006330FFF7B2FD00E0002004AB03EB850343F84A
S31508006340100C013500E00025032DE8D9002504AB23
S3150800635003EB850353F8106C26B131462046FFF748
S3150800636071FF00E00320012802D90135032DEED97B
S31508006370042800F0DB80012800F2DA8004F13B00F3
S31508006380FFF784FDB0F5007F40F0D48004F14600A5
S31508006390FFF77CFD804620B904F15400FFF77CFD29
S315080063A08046C4F8188094F8409084F8029009F161
S315080063B0FF33DBB2012B00F2BF8008FB09F994F822
S315080063C03D506581002D00F0B9806B1E1D4240F0DE
S315080063D0B78004F14100FFF759FD8246208110F08D
S315080063E00F0F40F0AF8004F14300FFF74FFD07465B
S315080063F020B904F15000FFF74FFD074604F13E00AF
S31508006400FFF744FD0346002800F09E8009EB0002D2
S3150800641002EB1A129742C0F09980BF1AB7FBF5F53E
S31508006420002D00F0958040F6F5718D4201D80127C0
S3150800643000E002274FF6F5718D4200D90327023591
S315080064406561E661334423623244A262032F0FD1A9
S3150800645004F15A00FFF71AFD00287BD1BAF1000FA4
S315080064607AD104F15C00FFF717FD6062AD000EE01B
S31508006470BAF1000F72D04B446362022F01D16D004E
S3150800648005E005EB450305F0010505EB530505F2A7
S31508006490FF15B8EB552F63D34FF0FF332361E36045
S315080064A080232371032F2CD104F16000FFF7EEFC43
S315080064B0012826D1711C2046FFF7AAFE08BB002337
S315080064C0237104F22E20FFF7E1FC4AF65523984281
S315080064D017D104F13000FFF7DFFC244B984210D1A6
S315080064E004F50570FFF7D8FC214B984209D104F54D
S315080064F00670FFF7D1FC206104F50770FFF7CCFCA6
S31508006500E06027701B4A138801339BB21380E3802F
S31508006510002026E00B2024E00C2022E0002020E0CA
S315080065200A201EE003201CE00A201AE0012018E0D9
S315080065300D2016E00D2014E00D2012E00D2010E0CD
S315080065400D200EE00D200CE00D200AE00D2008E0DD
S315080065500D2006E00D2004E00D2002E00D2000E0ED
S315080065600D2004B0BDE8F087841A0020525261411C
S3150800657072724161801A0020F8B50668012951D95E
S315080065807369994250D20C463378022B2AD0032BD2
S3150800659037D0012B4AD101EB5105316A01EB552160
S315080065A03046FFF735FE002842D16F1CC5F30805B3
S315080065B0354495F83050316A01EB57213046FFF7DC
S315080065C027FE002837D1C7F308073E4496F830005F
S315080065D045EA002014F0010F01D00009F8BDC0F308
S315080065E00B00F8BD316A01EB14213046FFF710FEA7
S315080065F020BB600000F4FF7030303044FFF746FCE3
S31508006600F8BD316A01EBD4113046FFF701FEC0B977
S31508006610A00000F4FE7030303044FFF73DFC20F057
S315080066207040F8BD0120F8BD0120F8BD0120F8BD75
S315080066304FF0FF30F8BD4FF0FF30F8BD4FF0FF3098
S31508006640F8BD4FF0FF30F8BD2DE9F0410768B1F508
S31508006650001F3DD206460C4611F01F0F3BD1316193
S3150800666085681DB93B78022B00D97D6A35B93B8907
S31508006670B3EB541F32D97B6AB3611AE0B7F80A80C4
S315080066804FEA48280EE029463046FFF775FF0546CB
S31508006690B0F1FF3F25D0012826D97B69984226D23A
S315080066A0C8EB04044445EED229463846FFF736FCC3
S315080066B0B0617561B369EBB103EB5423B36107F1BC
S315080066C03003C4F308042344F3610020BDE8F081D5
S315080066D00220BDE8F0810220BDE8F0810220BDE875
S315080066E0F0810120BDE8F0810220BDE8F08102209A
S315080066F0BDE8F0810220BDE8F08100BF2DE9F8432E
S31508006700012979D94369994278D217460C46054634
S315080067100378022B44D0032B54D0012B70D101EB04
S315080067205108016A01EB5821FFF772FD0646002859
S3150800673067D108F10109C8F3080814F001040BD061
S3150800674005EB080393F830203B0103F47F6302F05E
S315080067500F021343DBB200E0FBB2A84488F83030DE
S315080067600123EB70296A01EB59212846FFF750FDF2
S315080067700646002845D1C9F3080914B1C7F307121C
S3150800678008E005EB090393F8303023F00F03C7F34D
S3150800679003221A43A94489F830200123EB7030E01C
S315080067A0016A01EB1421FFF733FD064648BB60007A
S315080067B000F4FF703030B9B22844FFF779FB0123A3
S315080067C0EB701EE0016A01EBD411FFF721FD0646C6
S315080067D0B8B927F07047A40004F4FE7430342C448A
S315080067E02046FFF759FB00F0704139432046FFF772
S315080067F063FB0123EB7004E0022602E0022600E0B8
S3150800680002263046BDE8F8832DE9F04107460668BA
S31508006810884629B9F5687DB173699D420ED20EE0A6
S31508006820FFF7AAFE012846D9B0F1FF3F51D0736998
S3150800683098424ED3454602E0012500E001252C4644
S31508006840013473699C4202D3012D37D902242146AB
S315080068503846FFF791FE38B1012832D0B0F1FF3F34
S3150800686031D0AC42ECD130E04FF0FF322146304611
S31508006870FFF744FF034640B9B8F1000F05D022469A
S3150800688041463046FFF73AFF034673B9F460336969
S315080068907269023A934201D2013B3361337943F07C
S315080068A0010333712046BDE8F081012B10D14FF06A
S315080068B0FF30BDE8F0810120BDE8F0810020BDE889
S315080068C0F081BDE8F081BDE8F0810020BDE8F081E7
S315080068D00120BDE8F08100BFF8B50E46046801291D
S315080068E02CD90746114663699E4229D22AB14FF030
S315080068F0FF322046FFF702FF20BB31463846FFF736
S315080069003BFE0546F8B101281FD0B0F1FF3F1ED067
S31508006910002231462046FFF7F1FED0B92369B3F1CC
S31508006920FF3F05D001332361237943F00103237127
S3150800693063692E469D42E0D30020F8BD0220F8BDCB
S315080069400220F8BDF8BD0020F8BD0220F8BD0120E0
S31508006950F8BDF8BD2DE9F8430668036903F120057B
S315080069608369002B6ED0B5F5001F6ED288460446A3
S31508006970C5F30807002F5DD101338361416941B929
S315080069803389B3EB551F55D8002383610420BDE82E
S31508006990F8837389013B13EA55234BD1FFF7ECFDC6
S315080069A08146012854D9B0F1FF3F54D07369984203
S315080069B039D3B8F1000F04D10023A3610420BDE840
S315080069C0F88361692046FFF71FFF8146002845D0F6
S315080069D0012846D0B0F1FF3F46D03046FFF7EEFB20
S315080069E0002844D14FF40072002106F13000FFF769
S315080069F077FA49463046FFF791FAF0624FF00008F9
S31508006A000AE00123F3703046FFF7D8FB90BB08F184
S31508006A100108F36A0133F36273899845F1D3F36A7F
S31508006A20C8EB0303F362C4F8149049463046FFF7EF
S31508006A3075FAA061256107F130084644E661002031
S31508006A40BDE8F8830420BDE8F8830420BDE8F88390
S31508006A500220BDE8F8830120BDE8F8830720BDE8D9
S31508006A60F8830220BDE8F8830120BDE8F8830120F9
S31508006A70BDE8F8830120BDE8F88300BFF8B50446F1
S31508006A800F4606680021FFF7DFFD0246B8B9002564
S31508006A90A1693046FFF7BCFB024680B9E3691B785B
S31508006AA0E52B00D01BB90135BD4201D107E0002511
S31508006AB001212046FFF74EFF02460028E8D0042AA7
S31508006AC000D107221046F8BD2DE9F843044688464A
S31508006AD007684FF0FF094E4604254CE03846FFF795
S31508006AE097FB054600284BD1E1690A78002A46D06B
S31508006AF0CB7A03F03F03A371E52A2BD02E2A2BD09D
S31508006B0023F02000082814BF00200120404525D185
S31508006B100F2B15D112F0400F06D091F80D9002F008
S31508006B20BF02236963621646B24219D14B7B994567
S31508006B3018D1A06AFFF722FAB0B1013EF6B214E006
S31508006B4026B90846FFF7E8FA814519D04FF0FF3312
S31508006B50636215E0FF2608E0FF2606E0FF2604E04C
S31508006B60FF2602E0FF2600E0FF2600212046FFF769
S31508006B70F1FE054620B9A1690029AFD100E0042538
S31508006B800DB10023A3612846BDE8F88370B5044615
S31508006B9005680669416AB1F1FF3F03D0FFF754FD66
S31508006BA0034600E00023BBB9A1692846FFF730FB7E
S31508006BB0034670B9E269E52111700122EA7022697B
S31508006BC0964206D900212046FFF7C4FE0346002850
S31508006BD0EAD0042B00D10223184670BD2DE9F04FE8
S31508006BE083B006468A46D1F80090856A0024234673
S31508006BF05F1C19F803001F2805D92F2803D05C2825
S31508006C000AD100E0013709EB070219F807302F2BE4
S31508006C10F8D05C2BF6D017E0FE2C00F2E2800121BA
S31508006C2000F0D6FF8046002800F0DD807F2806D8D1
S31508006C3001467148FFF76AF9002840F0D68025F822
S31508006C4014803B460134D3E7CAF800201F2802D82F
S31508006C504FF004080CE04FF0000809E004F1004387
S31508006C60013B35F81330202B01D02E2B02D1013CE5
S31508006C70002CF3D1002325F81430002C00F0B7803F
S31508006C800B222021306AFFF72BF9002300E001339D
S31508006C9035F81320202AFAD02E2AF8D01BB148F04E
S31508006CA0030800E0013C6CB104F10042013A35F8F2
S31508006CB012202E2AF6D14FF0080B4FF0000ACDF815
S31508006CC004A005E04FF0080B4FF0000ACDF804A029
S31508006CD003F1010935F81370002F57D0202F03D080
S31508006CE02E2F05D14C4503D048F003084B46EFE755
S31508006CF0DA4501D24C4515D1BBF10B0F02D148F04C
S31508006D00030843E04C4501D048F003084C453DD301
S31508006D10019B9B00DBB2019323464FF00B0B4FF010
S31508006D20080AD5E77F2F0BD90021384600F050FF17
S31508006D30074618B1A0F18007304BDF5D48F002081E
S31508006D4027B139462E48FFF7E1F818B148F003088D
S31508006D505F2714E0A7F141039BB2192B04D8019BC6
S31508006D6043F0020301930AE0A7F161039BB2192BD2
S31508006D7005D8019B43F001030193203FBFB2336A54
S31508006D8003F80A704B460AF1010AA1E7336A1A7832
S31508006D90E52A01D105221A70BBF1080F03D1019B20
S31508006DA09B00DBB20193019901F00C020C2A03D077
S31508006DB001F00303032B01D148F0020818F0020F73
S31508006DC00AD1019B03F00303012B01D148F01008F7
S31508006DD0042A01D148F00808336A83F80B8000209A
S31508006DE006E0062004E0062002E0062000E0062071
S31508006DF003B0BDE8F08F00BF90910008A491000889
S31508006E009C910008F8B500238B758369002B69D01F
S31508006E100D460646436AB3F1FF3F17D0836A00243E
S31508006E2009E0002100F0D4FE50B1FE2C0AD82A1938
S31508006E3090753B4601349F1C18880028F1D102E062
S31508006E40002400E000242C440023A375AC7D002216
S31508006E50134628E0F069591CC35C202B22D0052B69
S31508006E6000D1E523092907D114B9A8182E27877553
S31508006E70A8182E2747720132A81843728CB9A3F1B5
S31508006E804100C0B219280AD8F069007B082901D93F
S31508006E90102700E00827074201D02033DBB2A818E4
S31508006EA0837501320B460A2BD4D934B9AB180021A5
S31508006EB09975F3691B7B03B90A462A440023537262
S31508006EC0F369DB7A2B72F0691C30FEF7E5FF286060
S31508006ED0F0691830FEF7DAFFA880F0691630FEF779
S31508006EE0D5FFE880F8BD00BF2DE9F0478146884602
S31508006EF001F11A00FEF7CAFFA8BB98F8005005F082
S31508006F003F056B1E03EB430503EB850501270024AC
S31508006F101BE01F4B185D4044FEF7B8FF06467FB1DD
S31508006F20FE2D23D800F072FE074605F1010A39F84E
S31508006F30150000F06BFE87421BD13746554603E025
S31508006F404FF6FF73984217D101340C2CE1D998F803
S31508006F50003013F0400F12D0A7B139F81530A3B995
S31508006F600120BDE8F0870020BDE8F0870020BDE8D5
S31508006F70F0870020BDE8F0870020BDE8F0870120F3
S31508006F80BDE8F0870120BDE8F0870020BDE8F0875E
S31508006F90249200082DE9F8430446D0F80080002121
S31508006FA0FFF752FB00285CD14FF0FF3363624FF0C6
S31508006FB0FF094F46A1694046FFF72AF90646002809
S31508006FC051D1E5692B78002B4FD0E97A01F03F02C1
S31508006FD0A271E52B04D011F0080F06D00F2A04D0B1
S31508006FE04FF0FF336362FF2733E00F2A17D1A06AF9
S31508006FF078B313F0400F06D095F80D9003F0BF0351
S31508007000226962621F46BB421ED16B7B99451DD120
S315080070102946FFF769FFD8B1013FFFB219E027B942
S315080070202846FFF779F8814522D0216ACB7A13F0F2
S31508007030010F04D10B222846FEF758FFD8B14FF0AE
S31508007040FF336362FF2704E0FF2702E0FF2700E023
S31508007050FF2700212046FFF77DFC0028AAD0BDE8BF
S31508007060F883BDE8F883BDE8F8830420BDE8F88313
S315080070703046BDE8F8833046BDE8F88330B583B0BE
S3150800708004460191056801E001330193019B1A78D2
S315080070902F2AF9D05C2AF7D00022A2601B781F2B72
S315080070A008D8236A8022DA7200212046FFF7CCFA34
S315080070B0034626E001A92046FFF790FD034600BBDC
S315080070C02046FFF767FF236ADA7A034628B10428C1
S315080070D017D112F0040F11D013E012F0040F10D1DB
S315080070E0A37913F0100F0BD02169C1F308013031D1
S315080070F029442846FEF71EFFA060DBE7052300E0CB
S315080071000523184603B030BD2DE9F04784B006685C
S31508007110D0F820A0D0F828809AF80B3013F0A00FEA
S3150800712040F08380002400E0013438F81430002B46
S31508007130FAD105460C22514601A8FEF7C7FE9DF86E
S315080071400F3013F0010F1ED000238AF80B30AB6204
S3150800715001270BE03B46424601A95046FEF78CFF45
S315080071602846FFF717FF814610B90137632FF1D973
S31508007170642F5CD0B9F1040F5BD19DF80F308AF803
S315080071800B30C5F828809DF80F3013F0020F06D093
S315080071900C342B4BA3FB0434A408013400E001246F
S315080071A021462846FFF76AFC034618BB013C21D056
S315080071B02969A1EB44112846FFF746FA0346C8B9E0
S315080071C0286AFEF7A9FF0746A9693046FFF720F89F
S315080071D0034678B93B46E2B2E969A86AFEF714FFA6
S315080071E00123F37000212846FFF7B4FB034608B9CC
S315080071F0013CE9D1FBB9A9693046FFF709F8814690
S31508007200D8B920220021E869FEF76AFE0B22296A0E
S31508007210E869FEF75BFEEA692B6ADB7A03F0180376
S3150800722013730123F370484607E0062005E007209C
S3150800723003E0484601E01846FFE704B0BDE8F087DA
S315080072404FECC44E70B50446FEF7B8FF0546002855
S3150800725037D12378032B2DD12379012B2AD104F199
S3150800726030064FF4007200213046FEF739FE4AF622
S31508007270552104F22E20FEF71BFE13493046FEF771
S315080072801BFE124904F50570FEF716FE216904F582
S315080072900670FEF711FEE16804F50770FEF70CFEAE
S315080072A0E2690132E262012331466078FCF71CFD8F
S315080072B000232371002211466078FCF741FD00B1D6
S315080072C00125284670BD00BF525261417272416164
S315080072D010B584B001900091144604A840F8041D26
S315080072E0FEF728FF002816DB0E4B53F820300BB1AB
S315080072F000221A70019B0BB100221A70019B094AE1
S3150800730042F820304BB1012C09D1002201A9684668
S31508007310FEF7C8FF04E00B2002E0002000E0002092
S3150800732004B010BD841A00202DE9F04393B00191F2
S31508007330002800F0AA80054616460023036002F0DE
S315080073401F073A4606A901A8FEF7ACFF002840F039
S315080073509E80069B079303AB0F934F4B119301999E
S3150800736007A8FFF78BFE044628B90F9B93F90B3045
S31508007370002B00DA062416F01C0F53D044B1042C57
S3150800738003D107A8FFF7C0FE044647F008070BE03D
S315080073909DF8223013F0110F03D116F0040F02D115
S315080073A002E0072400E00824002C4BD117F0080F50
S315080073B048D03A4E31460E980E30FEF77DFD3146DE
S315080073C00E981630FEF778FD20220E9BDA72069E7E
S315080073D0DDF8388041463046FEF7ACFD814600228E
S315080073E041463046FEF7B8FD00210E981C30FEF7E0
S315080073F063FD0122069BDA70B9F1000F22D0069BC5
S31508007400DE6A0022494607A8FFF766FA0446C8B9A5
S3150800741031460698FEF7FCFE044609F1FF33069A44
S31508007420D3600FE074B99DF8223013F0100F06D11F
S3150800743016F0020F06D013F0010F02D102E0042461
S3150800744000E007244CB917F0080F01D047F02007D1
S31508007450069BDB6A2B620E9B6B62CCB9069EDDF837
S31508007460388041463046FEF765FDA86008F11C00E5
S31508007470FEF712FDE86000236B746B61EB612F74F5
S315080074802E60F388AB80204603E0092001E000E087
S31508007490204613B0BDE8F08380180020000061483C
S315080074A02DE9F04F83B00446884615461F4600234B
S315080074B03B6001A9FEF768FE002840F0A280607CC8
S315080074C0002840F0A080237C13F0010F00F09A807A
S315080074D0E6686369F61AAE42C0F08E802E468BE0E7
S315080074E06369C3F30802002A70D1019A5289013AE6
S315080074F012EA532912D10BB9A06803E0A169204604
S31508007500FFF73AF8012802D8022060747BE0B0F150
S31508007510FF3F02D10120607475E0A061DDF804A088
S31508007520A1695046FEF7FAFC054610B902206074B8
S3150800753069E04D445FEA562B25D009EB0B03BAF8F0
S315080075400A20934201D9C9EB020B5B462A464146FB
S315080075509AF80100FCF79CFB10B10120607452E018
S31508007560237C13F0400F0BD0E069401B834507D9F5
S315080075704FF4007204F1280108EB4020FEF7A6FC40
S315080075804FEA4B2530E0E26995421ED0237C13F082
S31508007590400F0ED0012304F128019AF80100FCF7E8
S315080075A0A3FB10B1012060742DE0237C23F0400377
S315080075B0237401232A4604F1280101984078FCF730
S315080075C067FB10B1012060741DE0E5616169C1F3D4
S315080075D00801C1F50075AE4200D2354628312A4663
S315080075E021444046FEF772FCA84463692B44636154
S315080075F03B682B443B60761B002E7FF471AF00205E
S3150800760001E000E0072003B0BDE8F08F2DE9F04F58
S3150800761083B00446884616461F4600233B6001A9E8
S31508007620FEF7B2FD002840F0BE80607C002840F0DE
S31508007630BC80237C13F0020F00F0B6806369F34226
S31508007640C0F0A880DE43A5E06369C3F30802002AF8
S3150800765040F08180019A5289013A12EA53291DD1D4
S3150800766033B9A06840B900212046FFF7CDF803E0FA
S31508007670A1692046FFF7C8F8002800F08E80012887
S3150800768002D10220607490E0B0F1FF3F02D10120E0
S3150800769060748AE0A061A36803B9A060237C13F034
S315080076A0400F0FD00123E26904F1280101984078C0
S315080076B0FCF71AFB10B10120607476E0237C23F0F6
S315080076C040032374DDF804A0A1695046FEF726FCA2
S315080076D0054610B90220607467E04D445FEA562BF0
S315080076E025D009EB0B03BAF80A20934201D9C9EB56
S315080076F0020B5B462A4641469AF80100FCF7F4FA63
S3150800770010B10120607450E0E169491B8B450BD923
S315080077104FF4007208EB412104F12800FEF7D6FB6E
S31508007720237C23F0400323744FEA4B2525E0E369C5
S315080077309D420FD06269E3689A420BD201232A461A
S3150800774004F128019AF80100FCF7A2FA10B1012009
S3150800775060742AE0E5616069C0F30800C0F5007549
S31508007760AE4200D2354628302A4641462044FEF726
S31508007770ADFB237C43F040032374A84463692B4480
S315080077806361E268934238BF1346E3603B682B4463
S315080077903B60761B002E7FF457AF237C43F0200313
S315080077A02374002001E000E0072003B0BDE8F08F55
S315080077B070B582B004460E460A2902D10D21FFF79C
S315080077C0F7FF6368002B16DB5D1C23441E733C2DF4
S315080077D00DDD01AB2A4604F10C012068FFF716FF00
S315080077E0019B9D4201D1002501E04FF0FF35656000
S315080077F0A3680133A36002B070BD00BF30B583B083
S31508007800044601A9FEF7C0FC00283CD1227C12F0F0
S31508007810200F39D012F0400F0CD00123E26904F191
S31508007820280101984078FCF75FFA70BB237C23F0A7
S3150800783040032374216A0198FEF7EAFC38BB656A9F
S31508007840EB7A43F02003EB72A26829462068FEF71C
S3150800785083FBE16805F11C00FEF72EFB0D4905F1D7
S315080078601600FEF729FB002105F11200FEF720FBA2
S315080078700122019BDA700198FFF7E4FC237C23F0D0
S315080078802003237403E002E001E00120FFE703B0D0
S3150800789030BD00BF0000614810B582B00446FFF74E
S315080078A0ADFF034638B901A92046FEF76DFC03462D
S315080078B008B900222260184602B010BDF0B583B0A0
S315080078C004460E4601A9FEF75FFC002840F0A48096
S315080078D0657C002D40F0A180E368B34204D2227C87
S315080078E012F0020F00D11E46636900226261002E63
S315080078F05DD0019A57897F026BB1721EB2FBF7F20F
S31508007900013BB3FBF7F18A4205D37A421340636120
S31508007910F61AA16912E0A16879B92046FEF774FF44
S315080079200146012802D10220607479E0B0F1FF3FD8
S3150800793002D10120607473E0A060A16119BB002622
S3150800794038E0237C13F0020F05D02046FEF75CFFD3
S31508007950014620B91AE02046FEF70EFE0146B1F1AF
S31508007960FF3F02D1012060745AE0012903D9019B27
S315080079705B69994202D30220607451E0A161636990
S315080079803B446361F61BBE42DBD800E03E466369B2
S3150800799033446361C6F308035BB10198FEF7BEFA88
S315080079A010B9022060743BE000EB562602E0002680
S315080079B000E000266369C3F3080313B3E26996423D
S315080079C01FD0237C13F0400F0ED0012304F12801A9
S315080079D001984078FCF788F910B1012060741FE01F
S315080079E0237C23F0400323740123324604F1280143
S315080079F001984078FCF74CF910B1012060740FE04B
S31508007A00E6616369E268934209D9E360237C43F03F
S31508007A1020032374284603E002E0284600E02846AF
S31508007A2003B0F0BD30B591B001900D46002205A90E
S31508007A3001A8FEF737FC0446A8B902AB0D930B4B19
S31508007A400F93019905A8FFF719FB044658B90D9B32
S31508007A5093F90B30002B05DB2DB1294605A8FFF756
S31508007A60D1F900E00624204611B030BD8018002068
S31508007A7070B59CB00190022205A901A8FEF712FC78
S31508007A80059B1193044600284AD102AB1993264B4D
S31508007A901B93019911A8FFF7F1FA044600283FD174
S31508007AA0199B93F90B30002B05DB9DF84A3013F030
S31508007AB0010F02D102E0062400E00724ECB9059E76
S31508007AC018993046FEF736FA05469DF84A3013F0FF
S31508007AD0100F13D006960890002106A8FEF7B4FDED
S31508007AE0044658B9002106A8FEF7EEFF034600B97A
S31508007AF00723042B02D01C4600E0002584B911A8F0
S31508007B00FFF744F8044630B92DB10022294611A8DA
S31508007B10FEF7E2FE04461CB90598FFF793FB0446F8
S31508007B2020461CB070BD00BF801800202DE9F0412A
S31508007B3082B080460E4617460546002412E06B467C
S31508007B40012201A93846FFF7ABFC009B012B0ED199
S31508007B509DF804300D2B05D06A1C2B7001340A2BB6
S31508007B6004D01546731E9C42E9DB00E01546002347
S31508007B702B700CB9184600E0404602B0BDE8F0810B
S31508007B8010B594B00446019100230293039303E0D1
S31508007B90013401A8FFF70CFE21780029F8D1029AD2
S31508007BA0002A0BDB6B4604A90198FFF72FFD40B9A5
S31508007BB0009B029A9A4207D1039807E04FF0FF30DC
S31508007BC004E04FF0FF3001E04FF0FF3014B010BD75
S31508007BD07F2817D979B1FF2813D8A0F180030A4A5C
S31508007BE032F813007047084A32F81320904205D03D
S31508007BF001339BB200E000237F2BF4D98033D8B23F
S31508007C0070470020704700BFE4940008F0B4B0F550
S31508007C10805F01D2204B02E0204B00E02B461A88F9
S31508007C20002A36D0904234D31D1D5B88190ADBB270
S31508007C309C18A04228DA08292BD8DFE801F00509A4
S31508007C400F1215181B1E2100861A35F8160020E09B
S31508007C50821A02F00103C01A80B21AE0103880B204
S31508007C6017E0203880B214E0303880B211E01A38B4
S31508007C7080B20EE0083080B20BE0503880B208E0DF
S31508007C80A0F5E35080B204E00029C7D105EB430311
S31508007C90C5E7F0BC704700BFF092000834920008B0
S31508007CA010B4013A0A440BE00C784B7803EB042332
S31508007CB09BB2184480B2834201D9013080B20231A6
S31508007CC09142F1D307D10B781B02184480B2834244
S31508007CD001D9013080B25DF8044B704770B4C5789D
S31508007CE00D44EDB2134CE57083780E0A3344DBB2CB
S31508007CF0A37042786270007820709CB2A64206D9BA
S31508007D000132D2B20B4C62700AB901302070C9B286
S31508007D108D420CDA0133DBB2064A93703BB95378CD
S31508007D200133DBB2537013B913780133137070BC87
S31508007D30704700BFD829002010B5094C23680146B2
S31508007D4003F10800FFF7CAFF2368064A117819727B
S31508007D505178597291789972D278DA7210BD00BF4B
S31508007D60E4290020D82900200022124B1A7006E0C8
S31508007D700021114A22F8131001330E4A13700D4BD5
S31508007D801B78002BF4D000220A4B1A7008E06822F0
S31508007D900A4902FB0312002151760133054A137082
S31508007DA0044B1B78002BF2D04FF48062044B1A80E8
S31508007DB0704700BF921A0020502A0020E8290020A8
S31508007DC0901A002000220A4B1A700BE01946094A3D
S31508007DD032F813201AB9074B23F8110070470133FC
S31508007DE0034A1370024B1B78002BEFD0704700BF75
S31508007DF0921A0020502A0020030A43EA002080B283
S31508007E00704700BF08B5142205490020FFF748FF50
S31508007E1010B1FFF7F1FF08BD4FF6FF7008BD00BFB0
S31508007E206E2A002038B50D4D2C7C6B7C03EB0424A0
S31508007E30143CA4B22044082205F11A0180B2FFF7C7
S31508007E402FFF224605F12201FFF72AFF10B1FFF79F
S31508007E50D3FF38BD4FF6FF7038BD00BF602A00203B
S31508007E6008B50620FFF7DEFF08BD00BF70B5934BC7
S31508007E701C68934B934A1360934A136003280FD1E7
S31508007E80637E03F00F03032B40F02F85238A002B14
S31508007E9040F02B8508228D4B1A70FCF741FFEAE368
S31508007EA0022879D18A4AD3780133DBB2D37063B911
S31508007EB093780133DBB293703BB953780133DBB265
S31508007EC0537013B91378013313700023814A138052
S31508007ED0814A1380637E072B01D0052B0AD1A37E26
S31508007EE00133DBB2A376782B40F0FF840023637658
S31508007EF000F0FBBC002B00F0F884228A002A40D050
S31508007F00A27E511EA176002A40F0EF84E27E082A5E
S31508007F1005D0591EC9B201290ED8052A0CD100234D
S31508007F2063768022694B1A70FCF7FAFE14226B4BB3
S31508007F3083F82F2000F05BBC042A03D80321914064
S31508007F40C9B200E03021A1760132E27603F00F03D0
S31508007F50013B072B00F2C984DFE813F0BE010800D5
S31508007F600D003803C7043803C704380300225B4BE7
S31508007F7083F82F20B4E10422544B1A70FCF7D0FE84
S31508007F80AEE303F00F03032B40F0AF8408224F4BF8
S31508007F901A70FCF7C5FE6EE3504B9B7B452B40F0F1
S31508007FA0A4844E4A157C537C03EB0521494A128862
S31508007FB0914200F39A848DB2464B1D80474B1B7D38
S31508007FC013F03F0F40F09184444B5B7D002B40F04B
S31508007FD08C84434B1C880CB95B885BB13F4BDB8BAD
S31508007FE09C4240F082843D4B1A8C3D4B5B889A42FA
S31508007FF040F07B84FFF706FF4FF6FF73984240F088
S315080080007484364BDB7D062B23D0012B40F06D8420
S31508008010324B93F82230082B40F067842F4B00220E
S3150800802083F822209B8C4FF6F672934203D90933C4
S315080080302A4A938402E00833284A9384274B5A8BAA
S31508008040DA839A8B1A845C83254A52889A8300F0CD
S3150800805048BCFFF705FF4FF6FF73984240F045848A
S31508008060204C17E0617EA1B11C4B9A8CA3889A42DA
S315080080700FD11A4B5A8CE3889A420AD1174B5A8B5E
S3150800808023889A4205D1154B9A8B63889A4200F049
S3150800809041816834134B9C42E4D9104B93F82F3036
S315080080A003F03F03022B2FD10C4B9B8C99B20E4A3F
S315080080B0138000220D4B1A7022E000BFE42900202D
S315080080C0962A0020E0290020D4290020DC29002057
S315080080D08C1A0020D0290020A2300020602A002017
S315080080E05C2A0020E8290020881A0020921A00201D
S315080080F0924A32F8132091425BD00133904A1370AA
S315080081008F4B1B78002BF3D08E4B93F82F3013F040
S31508008110040F40F0EA838B4B142283F82F20282182
S31508008120894A1180502283F82E2093F8290093F863
S315080081302D2083F8292093F8281093F82C2083F80B
S31508008140282083F82C1093F8272093F82B4083F8DF
S31508008150274083F82B2093F82640794D2C7093F806
S315080081602A5083F8265083F82A400130C0B283F893
S315080081702D0068B94B1CDBB2724981F82C303BB92B
S31508008180531CDBB281F82B3013B9013481F82A402D
S315080081906C4B5A8C6D490A80998C59849A845A8BEF
S315080081A0DA839A8B1A846A4A1188598352889A8381
S315080081B06FE30024624B1C701CE019466822654870
S315080081C002FB0302527E1AB9682404FB010415E077
S315080081D0072A0CD13CB168225E4902FB0312917E44
S315080081E0A27E914203D95B4A682404FB0324013327
S315080081F0534A1370524B1B78002BDED0002C00F02C
S315080082007483554B1C600323A37623760023A3753A
S315080082100422E275E3764B4DAB8CA3806B8CE3802E
S315080082206B8B2380AB8B6380012060764B4B1A786F
S3150800823022735A7862739A78A273DB78E373208282
S3150800824095F82930E37295F82830A37295F8273007
S31508008250637295F826302372FFF76EFD95F82E00A7
S3150800826000F0F003502B37DD0022354B1A702BE057
S3150800827003F13602334DAA5C72B3012A03D10133E6
S315080082802F4A137020E0022A16D103F137022D4D2A
S31508008290AA5C042A10D101F13803EA5C39316B5C17
S315080082A043EA0222294B1A8040F20A63934228BF06
S315080082B013466382A3820FE003F1370221498A5CE1
S315080082C052B113441E4A13701D4B1B7819460209F6
S315080082D0053AB3EB820FCBDB10221A4B83F82F201B
S315080082E0184B93F82F2042F0020283F82F2002221F
S315080082F083F83620042283F83720062283F83820AC
S315080083000A2283F839202C210F4A1180602283F82B
S315080083102E2073E2104B1C600022114B1A70094B79
S3150800832093F82F2012F0040F1CD000236376202226
S315080083300B4B1A70FCF7F4FCD7E200BF502A00205A
S31508008340921A0020602A0020D0290020881A0020CE
S315080083505C2A0020E8290020E42900208C1A002045
S31508008360DC2900209C4B93F82E301B099B009B4868
S315080083700370EB1A143B9BB29948038001F00F0176
S31508008380022903D102F03F0112290FD013B912F0C6
S31508008390030F0BD0904BD98C2389994240F0238246
S315080083A08D4B198D6389994240F01D8212F0100F8A
S315080083B047D0218A002944D004F10C00FFF78EFC2F
S315080083C0854B93F82A30874A1078834239D1824BF5
S315080083D093F82B3051788B4233D17F4B93F82C305E
S315080083E0927893422DD17C4B93F82D507D4BDB78B8
S315080083F09D4226D120736173A273E373E37ECBB9E2
S31508008400237EA27E9B1ADBB2A17DA3EBD103DBB24E
S315080084105AB21944C9B2A175002A01DA5B425AB2A6
S31508008420E37DA2EB930253FA82F2D3B2E37503EB30
S31508008430D103237601226C4B1A70237EA376002380
S315080084402382617E01F00F03013B072B00F24D8268
S31508008450DFE813F00800230096007301A201BE01AD
S31508008460C9016501604B1B7813F0010F00F03D82CE
S315080084700323637640225C4B1A7000232382584BF1
S31508008480188820B14222584B1A70FFF755FC002273
S31508008490564B1A80FCF744FCEDE0534B1B7813F05F
S315080084A0010F63D04C4B93F82F3003F03F03122B88
S315080084B05CD1494B93F82E0000F0F003502B37DDC2
S315080084C00022464B1A702BE003F13602424DAA5C95
S315080084D072B3012A03D10133404A137020E0022AFD
S315080084E016D103F137023C4DAA5C042A10D101F1DA
S315080084F03803EA5C39316B5C43EA02223C4B1A804A
S3150800850040F20A63934228BF13466382A3820FE0B0
S3150800851003F1370230498A5C52B113442F4A13706B
S315080085202E4B1B7819460209053AB3EB820FCBDBB3
S3150800853003236376284B93F82620227293F8272084
S31508008540627293F82820A27293F82930E372012008
S31508008550FFF7F2FB4222244B1A7000232382204A9B
S315080085601380224A1380FCF7DBFB84E020221E4B93
S315080085701A70FCF7D5FB1F4B1B6800225A76C3E519
S31508008580154B93F82F3013F0010F35D011F0100F5B
S3150800859032D1238A002B40F0A881114D288801305A
S315080085A080B2FFF7C9FB104A137843F01003137023
S315080085B02A881AB143F002030B4A1370FCF7B0FB82
S315080085C001232382082363760023E3761122024BD4
S315080085D083F82F200BE100BF602A0020921A0020A2
S315080085E0D0290020D8290020DC290020A23000202C
S315080085F0881A0020E429002013F0200F10D099488B
S3150800860090F834301A0290F8353043EA0200964D55
S315080086102E6830442860954813430288D31A03808D
S31508008620924B188848B111F0100F06D1904A13786A
S3150800863043F002031370FFF77FFB8A4A92F8301063
S3150800864092F8313003EB01239BB28A4A1380A28A3F
S31508008650934200D80BB9874B1A80864B1B886382D6
S31508008660834B1B7813F0030F00F03F810022824BE7
S315080086701A80FCF755FB7E4B1B7813F0200F08D0A9
S3150800868000237D4A138063761422764B83F82F20C5
S31508008690ADE013F0100F0CD00023774A13800122A7
S315080086A0228204226276E37611226E4B83F82F200B
S315080086B09DE0714A12888AB113F0010F01D0002398
S315080086C02382238A43B9638A9A4201D96A4A138064
S315080086D0694B1B88238201E0674A13800023E376EF
S315080086E0664B1A68604B1A60634B1B884BB1238A2A
S315080086F03BB128335D4A138018225A4B83F82F2042
S3150800870078E05B4B1B7813F0020F00F0EE8028220E
S31508008710564B1A801022534B83F82F206AE0544B8D
S315080087201B7813F0010F00F0E08000236376102217
S315080087304F4B1A70FCF7F4FAD7E04C4B188808B17F
S31508008740FFF7FAFA474B93F82F3013F0010F15D0BD
S31508008750474B1B7813F0010F05D0072363760023D8
S31508008760A376238201E0062363760120FFF7E4FA65
S3150800877010223F4B1A70FCF7D3FA34E03C4B1B78B7
S3150800878013F0010F04D00523637600232382ACE09F
S31508008790364B1B883BBBA8E0344B188808B1FFF75B
S315080087A0CBFA304B93F82F3013F0010F0CD0072378
S315080087B063760023A3760120FFF7BEFA10222C4B1E
S315080087C01A70FCF7ADFA0EE0284B1B885BB98CE0F3
S315080087D0274B1B7813F0010F00F087800723637679
S315080087E00023A37681E010221E4B83F82F2028222F
S315080087F01E4B1A8050221B4B83F82E20227A194BC7
S3150800880083F82A20627A83F82B20A27A83F82C2010
S31508008810E27A83F82D20227B83F82620627B83F870
S315080088202720A27B83F82820E27B83F829200622CA
S31508008830DA75A2885A84E2889A84114A118859837B
S3150800884052889A832288DA8362881A84637E13F0B0
S31508008850100F17D0034B002283F8312083F83020FD
S3150800886017E000BF602A0020E0290020D029002058
S31508008870DC290020881A0020A2300020D4290020F4
S315080088805C2A00201C4B062283F830200A2283F833
S315080088903120194C4023A375184B1B881A0A2274D9
S315080088A06374002584F8355084F8345084F83250BF
S315080088B084F83350FFF7D4FAC04360864523A37380
S315080088C0E573657525750E4A138801339BB21380C7
S315080088D01A0AA274E37425766576FFF793FAC043FD
S315080088E020830022074B1A7070BD0023034A1380A9
S315080088F0044A137070BD00BF602A0020D0290020EA
S315080089008A1A0020DC29002000290CDD08B58AB265
S31508008910054B1A80054B1B68834203D0014618464F
S3150800892000F03CFA08BD7047A2300020D429002088
S31508008930F0B400223A4B1A701EE03A4D5A001A4417
S3150800894094002E192C5BA4B103EB4305AA00354D00
S315080089502A4452886AB10588AC420AD14488A242A0
S3150800896007D10C687460898831812F4A1278B272EF
S3150800897054E001332A4A1370294B1B78072BDCD99C
S315080089800022274B1A700FE0264D5A001A4494000D
S315080089902E192A5B2AB903EB4304A2002A445288FB
S315080089A032B101331E4A13701D4B1B78072BEBD9C6
S315080089B0082B28D100231D4A13701D4A1370184A24
S315080089C0137013E0184A147803EB4305AA00154DF3
S315080089D02A44927AA61A154D2D78AE4203DD134A1B
S315080089E01670134A137001330D4A13700C4B1B781B
S315080089F0072BE7D90E4B1B78094A137003EB430381
S31508008A009A00084E16440268334643F8042B0A684F
S31508008A1072608A889A80044B1B78B372F0BC7047E0
S31508008A209A1A00209C1A0020FD1A00209B1A002082
S31508008A30FC1A002010B4154B1C780134E4B21C70E3
S31508008A400022134B1A7019E012485A001A44910072
S31508008A504218415A52880A430DD003EB43018A0053
S31508008A600244927AA21A772A05DD03EB43018A00AB
S31508008A700020084988500133054A1370044B1B78B7
S31508008A80072BE1D95DF8044B704700BFFD1A00209B
S31508008A909A1A00209C1A002010B5324B1B88292BE5
S31508008AA003D800222F4B1A8010BD00222D4B1A80A6
S31508008AB02D4B9B8AB3F5807F03D0B3F5007F3FD05B
S31508008AC010BD294BDA8C294B1B889A4249D1264B73
S31508008AD01A8D264B5B889A4243D1254C2146A01D08
S31508008AE0FFF726FF002204F8022C022204F8012CC4
S31508008AF02168C4F80A10A188E1811E490868206027
S31508008B008988A18044F8100C24F80C1CD4F80A10A3
S31508008B1044F8161CE28924F8122CE288228222895B
S31508008B206282124A1188E18052882281082204F85A
S31508008B300A2C062204F8092C2A220A4B1A8010BD90
S31508008B40094BDA8C094B1B889A420AD1064B1A8DB7
S31508008B50064B5B889A4204D1054801460630FFF762
S31508008B60E7FE10BDD0290020602A00205C2A0020DC
S31508008B70762A0020941A002030B44C4BD98B8AB23E
S31508008B804FF6FF739A420CD1484B188C4FF6FF7379
S31508008B90984206D1454B464A1068186092889A80D2
S31508008BA072E0444B1B88444800885340184209D158
S31508008BB03E4B1A8C94B23F4B5B883F4840886340D3
S31508008BC0184206D03D4B3E4A1188198052885A8071
S31508008BD002E03A4B19805A8000223A4B1A7016E086
S31508008BE039485A001A4491004518344A1488425A9A
S31508008BF0944209D1314A508803EB43018A0032492D
S31508008C000A445288904206D001332E4A13702D4BDF
S31508008C101B78072BE4D9082B30D1244B4FF0FF32B1
S31508008C201A609A8000221A629A8428490868C3F84A
S31508008C30060089885981C3F8160059831F49088890
S31508008C40D884498819851B49088898834988D9830F
S31508008C501A75012159759A73D973082119745A74AA
S31508008C6006229A740422DA74197306225A73363362
S31508008C70174A13602A22174B1A8014E00B4B55F833
S31508008C80042F1A60AA889A80084B104A1168C3F8FC
S31508008C90061092885A8108221A7300225A730D4ABE
S31508008CA013880E33138030BC704700BF602A00203B
S31508008CB0E49500085C2A0020582A0020001B0020A2
S31508008CC0542A00209A1A00209C1A0020941A002080
S31508008CD0E0290020D029002008B5074B044613B127
S31508008CE00021AFF30080054B1868836A03B19847E3
S31508008CF02046F7F77FFF00BF00000000EC9500084C
S31508008D0070B50E4B0E4CE41AA41000251E46A5425B
S31508008D1004D056F8253098470135F8E700F05EF894
S31508008D20084C094BE41AA41000251E46A54204D097
S31508008D3056F8253098470135F8E770BDB802002087
S31508008D40B8020020BC020020B8020020034B1B68B2
S31508008D50186A034B002808BF1846704748010020C8
S31508008D604C01002008B5034B1868FFF7EFFFD0F851
S31508008D70EC0008BD4801002082B001B901A93AB14A
S31508008D8043B113780B601278101C18BF012003E05A
S31508008D90104601E06FF0010002B0704710B5431E9F
S31508008DA00A44914204D011F8014B03F8014FF8E741
S31508008DB010BD02440346934202D003F8011BFAE7AA
S31508008DC0704749B1FF2A85BF8A2303600A704FF0AE
S31508008DD0FF3098BF0120704708467047F8B500BFB6
S31508008DE0F8BC08BC9E467047F8B500BFF8BC08BC7E
S31508008DF09E4670476C69622F7569702F6E6574643C
S31508008E0065762E630000000057696E55534220426E
S31508008E10756C6B2044657669636500004F70656EF6
S31508008E20424C5420557365720000000030303030D3
S31508008E30303030303035304300000000446566611C
S31508008E40756C740057696E5553422042756C6B20D9
S31508008E50496E746572666163650000002F64656D0E
S31508008E606F70726F675F6F6C696D65785F73746D2D
S31508008E703332653430372E73726563002F626F6F35
S31508008E80746C6F672E74787400000000303A000026
S31508008E902E2E2F2E2E2F2E2E2F536F757263652F83
S31508008EA066696C652E6300004669726D7761726546
S31508008EB020757064617465207265717565737420B8
S31508008EC064657465637465640A0D00004F70656EA9
S31508008ED0696E67206669726D776172652066696C6E
S31508008EE06520666F722072656164696E672E2E2E24
S31508008EF0000000004552524F520A0D004F4B0A0D12
S31508008F00000000005374617274696E6720746865A6
S31508008F102070726F6772616D6D696E672073657117
S31508008F2075656E63650A0D0050617273696E672018
S31508008F306669726D776172652066696C6520746F03
S31508008F402064657465637420657261736520626C5C
S31508008F506F636B732E2E2E0045726173696E6720E0
S31508008F60000000002062797465732066726F6D20B8
S31508008F706D656D6F7279206174203078000000008D
S31508008F8052656164696E67206C696E652066726FEA
S31508008F906D2066696C652E2E2E4552524F520A0D6B
S31508008FA000000000496E76616C6964206368656339
S31508008FB06B73756D20666F756E642E2E2E45525234
S31508008FC04F520A0D0000000050726F6772616D6D96
S31508008FD0696E67200000000020627974657320744A
S31508008FE06F206D656D6F727920617420307800008E
S31508008FF057726974696E672070726F6772616D2047
S31508009000636865636B73756D2E2E2E00436C6F73E4
S31508009010696E67206669726D776172652066696C2C
S31508009020650A0D004669726D776172652075706410
S31508009030617465207375636365737366756C6C79A3
S3150800904020636F6D706C657465640A0D000000001E
S315080090504F70656E424C54002E2E2F2E2E2F2E2E1C
S315080090602F536F757263652F41524D434D345F53CD
S31508009070544D333246342F63616E2E630000000070
S3150800908005020602060307030803090309040A047E
S315080090900B040C040C050D050E050F050F0610062E
S315080090A0100710080000080010001800200028000B
S315080090B03000380040004800500058008000880002
S315080090C090009800A000A800B000B800C000C80032
S315080090D0D000D80000C000080040000003000000CF
S315080090E0000001080000010004000000000002085A
S315080090F0000002000500000000000408000002004D
S315080091000600000000000608000002000700000034
S3150800911000000808000002000800000000000A0815
S31508009120000002000900000000000C080000020010
S315080091300A00000000000E08000002000B000000F4
S315080091402E2E2F2E2E2F2E2E2F536F757263652FD0
S3150800915041524D434D345F53544D333246342F7587
S3150800916073622E63000000002E2E2F2E2E2F2E2E19
S315080091702F536F757263652F41524D434D345F53BC
S31508009180544D333246342F756172742E63000000D5
S31508009190222A3A3C3E3F7C7F000000002B2C3B3DB8
S315080091A05B5D0000809A45418E418F804545454963
S315080091B049498E8F9092924F994F555559999A9B36
S315080091C09C9D9E9F41494F55A5A5A6A7A8A9AAABB0
S315080091D0ACADAEAFB0B1B2B3B4B5B6B7B8B9BABB49
S315080091E0BCBDBEBFC0C1C2C3C4C5C6C7C8C9CACB39
S315080091F0CCCDCECFD0D1D2D3D4D5D6D7D8D9DADB29
S31508009200DCDDDEDFE0E1E2E3E4E5E6E7E8E9EAEB18
S31508009210ECEDEEEFF0F1F2F3F4F5F6F7F8F9FAFB08
S31508009220FCFDFEFF01030507090E10121416181C93
S315080092301E0000007D1D0100632C001E9601A01E65
S315080092405A01001F0806101F0606201F0806301FB1
S315080092500806401F0606511F0700591F521F5B1FAD
S31508009260541F5D1F561F5F1F601F0806701F0E00E4
S31508009270BA1FBB1FC81FC91FCA1FCB1FDA1FDB1F98
S31508009280F81FF91FEA1FEB1FFA1FFB1F801F0806AE
S31508009290901F0806A01F0806B01F0400B81FB91FB4
S315080092A0B21FBC1FCC1F0100C31FD01F0206E01F40
S315080092B00206E51F0100EC1FF21F0100FC1F4E21EC
S315080092C00100322170211002842101008321D0245B
S315080092D01A05302C2F04602C0201672C0601752C08
S315080092E00201802C6401002D260841FF1A030000A4
S315080092F061001A03E0001703F8000703FF000100E6
S3150800930078010001300132010601390110014A01D4
S315080093102E017901060180014D0043028101820177
S3150800932082018401840186018701870189018A01F6
S315080093308B018B018D018E018F01900191019101A5
S3150800934093019401F60196019701980198013D024F
S315080093509B019C019D0120029F01A001A001A20181
S31508009360A201A401A401A601A701A701A901AA01B6
S31508009370AB01AC01AC01AE01AF01AF01B101B20165
S31508009380B301B301B501B501B701B801B801BA0116
S31508009390BB01BC01BC01BE01F701C001C101C2018C
S315080093A0C301C401C501C401C701C801C701CA0177
S315080093B0CB01CA01CD011001DD0101008E01DE01DC
S315080093C01201F3010300F101F401F401F801280187
S315080093D0220212013A020900652C3B023B023D02B9
S315080093E0662C3F0240024102410246020A0153022C
S315080093F0400081018601550289018A0158028F01C0
S315080094005A0290015C025D025E025F0293016102EC
S315080094106202940164026502660267029701960178
S315080094206A02622C6C026D026E029C017002710265
S315080094309D01730274029F0176027702780279020F
S315080094407A027B027C02642C7E027F02A6018102DC
S315080094508202A9018402850286028702AE014402BD
S31508009460B101B20145028D028E028F02900291026D
S31508009470B7017B030300FD03FE03FF03AC030400EF
S315080094808603880389038A03B1031103C203020012
S31508009490A303A303C4030803CC0303008C038E03AE
S315080094A08F03D8031801F2030A00F903F303F40340
S315080094B0F503F603F703F703F903FA03FA0330048F
S315080094C0200350041007600422018A043601C104EF
S315080094D00E01CF040100C004D0044401610526042E
S315080094E000000000C700FC00E900E200E400E0001C
S315080094F0E500E700EA00EB00E800EF00EE00EC000C
S31508009500C400C500C900E600C600F400F600F20073
S31508009510FB00F900FF00D600DC00A200A300A500AE
S31508009520A7209201E100ED00F300FA00F100D10056
S31508009530AA00BA00BF001023AC00BD00BC00A10001
S31508009540AB00BB009125922593250225242561258C
S315080095506225562555256325512557255D255C2504
S315080095605B251025142534252C251C2500253C258E
S315080095705E255F255A2554256925662560255025CB
S315080095806C2567256825642565255925582552259E
S3150800959053256B256A2518250C25882584258C25B1
S315080095A090258025B103DF009303C003A303C303FB
S315080095B0B500C403A6039803A903B4031E22C60371
S315080095C0B50329226122B1006522642220232123C2
S315080095D0F7004822B0001922B7001A227F20B200ED
S315080095E0A025A000FFFFFFFFFFFF0000E800002006
S315080095F04300504F534958002E00002020202020B9
S315080096002020202028282828282020202020202024
S315080096102020202020202020202020881010101014
S315080096201010101010101010101010040404040468
S315080096300404040404101010101010104141414194
S31508009640414101010101010101010101010101017C
S31508009650010101010101101010101010424242428E
S31508009660424202020202020202020202020202024C
S315080096700202020202021010101020000000000070
S3150800968000000000000000000000000000000000CC
S3150800969000000000000000000000000000000000BC
S315080096A000000000000000000000000000000000AC
S315080096B0000000000000000000000000000000009C
S315080096C0000000000000000000000000000000008C
S315080096D0000000000000000000000000000000007C
S315080096E0000000000000000000000000000000006C
S315080096F0000000000000000000000000000000005C
S30D08009700E46AFF7F0100000086
S3150800970804000020C905000815050008C504000856
S315080097182D0400089504000811040008F903000838
S315080097283D0400084D0400085D0400087504000897
S3150800973800000000010203040102030406070809E1
S315080097480100000001000000A53D0008B13D000821
S31508009758D93D0008BD3D0008F53D0008113E000842
S315080097682D3E0008040309041201100100000040F8
S31508009778501DAC600001010203010000F93E000813
S31508009788E13E0008813E00080000000000000000D5
S31508009798693E0008753E0008553E000800000000AE
S315080097A800000000493E000809022000010100C027
S315080097B8320904000002FF00000007058102400084
S315080097C8FF070501024000FF5141000855410008FE
S315080097D8594100085D410008654100086D410008C7
S315080097E8794100080400000000000000000000009D
S315080097F80000000000000000000000000000000053
S315080098080000000000000000000000000000000042
S315080098180000000000000000000000000000000032
S315080098280000000000000000000000000000000022
S315080098380000000000000000000000000000000012
S315080098480000000000000000E800002043000000B7
S3150800985800000000000000000000000000000000F2
S31508009868000000000000000000000000430000009F
S3150800987800000000000000000000000000000000D2
S31508009888000000000000000000000000430000007F
S3150800989800000000000000000000000000000000B2
S315080098A8000000000000000000000000430000005F
S315080098B80000000000000000000000000000000092
S315080098C8000000000000000000000000430000003F
S315080098D80000000000000000000000000000000072
S315080098E8000000000000000000000000430000001F
S315080098F80000000000000000000000000000000052
S3150800990800000000000000000000000043000000FE
S315080099180000000000000000000000000000000031
S31508009928000000000000000000000000C38D0008C9
S31508009938798D000800000000FA950008F8950008D7
S31508009948F9950008F9950008F9950008F9950008A9
S31508009958F9950008F9950008F9950008F995000899
S31508009968F9950008FFFFFFFFFFFFFFFFFFFFFFFF57
S31508009978FFFF000001004153434949000000000069
S3150800998800000000000000000000000000000000C1
S315080099980000000000004153434949000000000048
S315080099A800000000000000000000000000000000A1
S315080099B80000000000000000AD0100088901000849
S70508000000F2
